:020000040000FA
:060000006CEF2EF012006F
:020006001200E6
:0600080094EF13F012005A
:02000E00253893
:070010006C6400253564005B
:0600180062EF13F012007C
:02001E000100DF
:0C002000245D000000020000050100004B
:04002C00D9CFE6FF43
:10003000E1CFD9FFFE0EDB50A96EA69EA69CA6803E
:10004000F40EE66E010EE66EE66AE66AEBEC12F07E
:10005000E552E552E552E552A85000D0E552E7CF0F
:10006000D9FF1200D9CFE6FFE1CFD9FFFE0EDB505A
:10007000A96EFD0EDB50A86EA69EA684550EA76E37
:10008000AA0EA76EA682A1A8FED7A198A694E552B3
:10009000E7CFD9FF1200D9CFE6FFE1CFD9FFFB0EA2
:1000A000DBCFE9FFFC0EDBCFEAFFEF501AE0FB0EDF
:1000B000DBCFE9FFDB2AFC0EDBCFEAFF01E3DB2A23
:1000C000EF50E66EFD0EDBCF00F0DB2AFE0EDBCF3D
:1000D00001F001E3DB2A0050E66EC4DFE552E55291
:1000E000DED7E552E7CFD9FF1200D9CFE6FFE1CF47
:1000F000D9FF020EE126FD0EDBCFE6FF97DFE552CA
:10010000DE6EDD6AD9CFE9FFDACFEAFFEE50ED10FF
:1001100001E11ED0DFCFE6FF68D8E552FD0EDB2AF5
:10012000FE0E01E3DB2AFD0EDBCF00F0FE0EDBCF7F
:1001300001F0013404E20050FF08000E015401E216
:1001400007D0D9CFE9FFDACFEAFFEE50ED10D3E1C7
:10015000980EE66E3A0EE66EE66AE66AEBEC12F090
:10016000E552E552E552E552020EE15C02E2E16A37
:10017000E552E16EE552E7CFD9FF1200948E949CD0
:10018000200EAF6EAC8AAC84AC98AC9CAB8EAB9CB2
:10019000AB889E989E9A9D8AF28EF28C1200D9CFDF
:1001A000E6FFE1CFD9FFE65201010451021902E155
:1001B0000551031901E1F8D702C1E9FF03C1EAFFC4
:1001C000022B000E0323EFCFDFFF830E025D020E32
:1001D000035904E35B0E026F020E036FDF5000D081
:1001E000E552E552E7CFD9FF1200D9CFE6FFE1CFC4
:1001F000D9FF020EE126DE6ADD6AACB210D0DF2A3A
:10020000010E01E3DB2AD9CFE9FFDACFEAFF100EB6
:10021000D880EE54270EED5401E206D0EED7FE0E44
:10022000DB50AD6E9EA8FED7020EE15C02E2E16AF1
:10023000E552E16EE552E7CFD9FF1200D9CFE6FFD4
:10024000E1CFD9FF030EE126FD0EDBCFDEFFDBCFD2
:10025000DDFFA5DFE76E020EE7CFDBFFFC0EDB5014
:10026000F36E020EDB50F35C0DE0FD0EDBCFE9FF19
:10027000DB2AFE0EDBCFEAFF01E3DB2A020EDBCF37
:10028000EFFFE7D7FD0EDBCFE9FFFE0EDBCFEAFF86
:10029000EF6ADECF00F0DDCF01F000C0F3FF01C058
:1002A000F4FF030EE15C03E200D0E16AE552E16E87
:1002B000E552E7CFD9FF1200D9CFE6FFE1CFD9FF52
:1002C000020EE126DE6ADD6AFD0EDBCFE9FFFE0EDF
:1002D000DBCFEAFFEF5014E0FD0EDBCFE9FFFE0EAF
:1002E000DBCFEAFFEF50E66E80DFE552DF2A010E3A
:1002F00001E3DB2AFD0EDB2AFE0E01E3DB2AE4D755
:10030000010EF36EF46A020EE15C03E200D0E16AD2
:10031000E552E16EE552E7CFD9FF12000D0EE66E11
:1003200064DFE5520A0EE66E60DFE5521200D9CFB7
:10033000E6FFE1CFD9FFFE0EDB50000803E2FE0E20
:10034000DB06F9D7E552E7CFD9FF1200D9CFE6FF98
:10035000E1CFD9FFFE0EDBCFE6FF33EC2EF0E55206
:10036000E552E7CFD9FF1200D9CFE6FFE1CFD9FFA1
:10037000030EE126FE0EDB505F0801E26ED0FD0E9B
:10038000DB503F0801E269D0FE0EDBCFE6FFFD0E39
:10039000DB50F80BE842E842E842600DF350E552CA
:1003A000E724DE6EDD6AFD0EDBCFE6FFDB50F80BE7
:1003B000E842E842E842080DF350E552E75CE76E98
:1003C000020EE7CFDBFFFC0EDB5016E1010EF36EF1
:1003D000020EDB5004E0D890F336E806FCE1F3505F
:1003E000E81C006EDECFE9FFDDCFEAFF580EE926FC
:1003F000010EEA220050EF16FC0EDB0415E1010E9F
:10040000F36E020EDB5004E0D890F336E806FCE110
:10041000F350006EDECFE9FFDDCFEAFF580EE9268C
:10042000010EEA220050EF12FC0EDB50020815E12B
:10043000010EF36E020EDB5004E0D890F336E806AE
:10044000FCE1F350006EDECFE9FFDDCFEAFF580E8E
:10045000E926010EEA220050EF1A030EE15C02E2E7
:10046000E16AE552E16EE552E7CFD9FF1200D9CF3C
:10047000E6FFE1CFD9FF0A0EE126FB0EDBCFE6FF58
:10048000FD0EDB50E552E75CE66ED950020FE96ED7
:10049000DACFEAFFE552E750EE6EED6AFC0EDBCFF5
:1004A000E6FFFE0EDB50E552E75CDE6EDD6A020E13
:1004B000DBCF00F0030EDBCF01F00001800E011452
:1004C00015E020682168020EDBCF25F0030EDBCF9C
:1004D00026F0D0EC21F0020E1EC0DBFF030E1FC081
:1004E000DBFF060EDB68070EDB6807D0010EF36E3C
:1004F000060EF3CFDBFF070EDB6ADECF00F0DDCFA9
:1005000001F00001800E011411E020682168DECFA7
:1005100025F0DDCF26F0D0EC21F01EC0DEFF1FC09D
:10052000DDFF040EDB68050EDB6807D0010EF36EFD
:10053000040EF3CFDBFF050EDB6AD9CFE9FFDACF7C
:10054000EAFF010ED890EE36ED36E806FBE1D95011
:10055000020FE96EDACFEAFF010ED890EE36ED36E3
:10056000E806FBE1FA0EDBCFE6FFFD0EDBCFE6FF90
:10057000FE0EDBCFE6FFF8DEE552E552E552DECFB8
:1005800000F0DDCF01F0020EDBCF02F0030EDBCF77
:1005900003F003500118E8AE02D0013404D000503B
:1005A000025C0150035867E2DECF02F0DDCF03F0BA
:1005B000D89003320232020EDBCF20F0030EDBCFE5
:1005C00021F00250205C006E03502158016E080E8D
:1005D00000C0DBFF090E01C0DBFFFC0EDB50F36E39
:1005E000FE0EDB50F35C46E0080EDBCF00F0090E98
:1005F000DBCF01F00001800E011416E1FD0EDBCF10
:10060000E7FF060EDB50E726FD0EE7CFDBFFDECF70
:1006100000F0DDCF01F0D950080FE96EDACFEAFF24
:100620000050EE5E0150ED5AFE0EDBCFE7FF040EE8
:10063000DB50E726FE0EE7CFDBFF020EDBCF00F03C
:10064000030EDBCF01F0D950080FE96EDACFEAFFD5
:100650000050EE260150ED22FA0EDBCFE6FFFD0E34
:10066000DBCFE6FFFE0EDBCFE6FF7EDEE552E55296
:10067000E552B3D762D0020EDBCF02F0030EDBCF20
:1006800003F0D890033202320250DE5C006E035059
:10069000DD58016E080E00C0DBFF090E01C0DBFF54
:1006A000FB0EDB50F36EFD0EDB50F35C46E0080EF4
:1006B000DBCF00F0090EDBCF01F00001800E01144A
:1006C00018E1FE0EDBCFE7FF040EDB50E726FE0E3F
:1006D000E7CFDBFF020EDBCF00F0030EDBCF01F034
:1006E000D950080FE96EDACFEAFF0050EE5E0150F4
:1006F000ED5AFD0EDBCFE7FF060EDB50E726FD0EC1
:10070000E7CFDBFFDECF00F0DDCF01F0D950080FDF
:10071000E96EDACFEAFF0050EE260150ED22FA0E24
:10072000DBCFE6FFFD0EDBCFE6FFFE0EDBCFE6FF05
:100730001BDEE552E552E552B3D70A0EE15C02E258
:10074000E16AE552E16EE552E7CFD9FF1200D9CF59
:10075000E6FFE1CFD9FF020EE126E66AE66A50DA4B
:10076000E552E55202018B6B8C6BDE6ADD6ADECFEF
:1007700000F0DDCF01F0000E005C030E015811E225
:10078000DECFE9FFDDCFEAFF580EE926010EEA22AF
:10079000EF50E66EF3D9E552DF2A010E01E3DB2AC2
:1007A000E6D7020EE15C02E2E16AE552E16EE55253
:1007B000E7CFD9FF1200D9CFE6FFE1CFD9FFFA0E7C
:1007C000DBCFE6FFFD0EDBCFE6FFFC0EDBCFE6FF67
:1007D000FD0EDBCFE6FFFE0EDBCFE6FF48DE006E50
:1007E000050EE15E0050FA0EDBCFE6FFFB0EDBCF1D
:1007F000E6FFFC0EDBCFE6FFFD0EDBCFE6FFFC0ED7
:10080000DBCFE6FF34DE006E050EE15E0050FA0E2F
:10081000DBCFE6FFFB0EDBCFE6FFFE0EDBCFE6FF16
:10082000FB0EDBCFE6FFFC0EDBCFE6FF20DE006E2B
:10083000050EE15E0050FA0EDBCFE6FFFD0EDBCFCA
:10084000E6FFFE0EDBCFE6FFFB0EDBCFE6FFFE0E84
:10085000DBCFE6FF0CDE006E050EE15E005077DFB9
:10086000E552E7CFD9FF1200D9CFE6FFE1CFD9FF9C
:10087000050EE126030EDB6AFD0EDBCFE6FFFE0E62
:10088000DB50E552E75CE76E040EE7CFDBFFFC0EC2
:10089000DB50E76E020EE7CFDBFF030E006EFC0EAF
:1008A000DB50E824005CDE6EDD6A030EDBCF00F077
:1008B000020EDB50D880005401E2F3D0FB0EDBCFF8
:1008C000E6FF020EDBCFE6FFFD0EDB50E552E7242C
:1008D000E66E030EDBCFE6FFFE0EDB50E552E724AB
:1008E000E66E42DDE552E552E552FB0EDBCFE6FF58
:1008F000FD0EDBCFE6FF020EDB50E552E75CE66E55
:10090000030EDBCFE6FFFE0EDB50E552E724E66E7A
:100910002BDDE552E552E552FB0EDBCFE6FF020E82
:10092000DBCFE6FFFD0EDB50E552E724E66EFE0E60
:10093000DBCFE6FF030EDB50E552E75CE66E14DD2D
:10094000E552E552E552FB0EDBCFE6FFFD0EDBCFB5
:10095000E6FF020EDB50E552E75CE66EFE0EDBCFF3
:10096000E6FF030EDB50E552E75CE66EFDDCE55288
:10097000E552E552FB0EDBCFE6FF030EDBCFE6FFD1
:10098000FD0EDB50E552E724E66E040EDBCFE6FFFA
:10099000020EDBCFE6FFFD0EDB50E552E724E55209
:1009A000D880E754E66EE0DCE552E552E552FB0EF6
:1009B000DBCFE6FFFD0EDBCFE6FF030EDB50E5529B
:1009C000E75CE66E040EDBCFE6FF020EDBCFE6FF50
:1009D000FD0EDB50E552E724E552D880E754E66E81
:1009E000C3DCE552E552E552FB0EDBCFE6FF030E1A
:1009F000DBCFE6FFFD0EDB50E552E724E66E040E8A
:100A0000DBCFE6FFFD0EDBCFE6FF020EDB50E5524B
:100A1000E75CE552D880E754E66EA6DCE552E55285
:100A2000E552FB0EDBCFE6FFFD0EDBCFE6FF030E4C
:100A3000DB50E552E75CE66E040EDBCFE6FFFD0E11
:100A4000DBCFE6FF020EDB50E552E75CE552D880D3
:100A5000E754E66E89DCE552E552E552DECF00F060
:100A6000DDCF01F00001800E011409E0030EDB5020
:100A7000040DF350060FDE26000EDD220FD0030E0C
:100A8000DBCFE6FF020EDB50E552E75C040DF350CE
:100A90000A0FDE26000EDD22020EDB06030EDB2A25
:100AA00004D755DE050EE15C02E2E16AE552E16E33
:100AB000E552E7CFD9FF1200828282908294960E8F
:100AC000E66E44DCE55282808284640EE66E3EDC93
:100AD000E552210EE66E3DD8E552900EE66E39D80D
:100AE000E552050EE66E35D8E552130EE66E31D8A6
:100AF000E552200EE66E2DD8E552960EE66E26DC07
:100B0000E5520C0EE66E25D8E552320EE66E1EDC7E
:100B1000E55212008290E66AE66A72D8E552E55222
:100B200001013D6B3E6BD8903E5104E6000E3D5DE9
:100B3000030E3E590DE2E66A21D8E5520A0EE66E32
:100B400097EC01F0E55201013D2B000E3E23EBD75F
:100B50001200D9CFE6FFE1CFD9FF82928290190E21
:100B6000E66E97EC01F0E552FE0EDBCFE6FF1BD8F8
:100B7000E5528280E552E7CFD9FF1200D9CFE6FFD8
:100B8000E1CFD9FF82828290190EE66E97EC01F0D8
:100B9000E552FE0EDBCFE6FF06D8E5528280E55235
:100BA000E7CFD9FF1200D9CFE6FFE1CFD9FFE65258
:100BB000080EDF6EDFCF00F0000EE76E0018E8AE23
:100BC00002D0003403D0E750D880005414E282965B
:100BD0000A0EE66E97EC01F0E552FE0EDBBE02D087
:100BE000829801D082888286DB50020DFE0EF3CF00
:100BF000DBFFDF06DFD7E552E552E7CFD9FF120072
:100C0000D9CFE6FFE1CFD9FFFD0EDB50070B40093E
:100C1000E66E9FDFE552FE0EDB507F0B8009E66E2D
:100C200098DFE552E552E7CFD9FF1200D9CFE6FFB2
:100C3000E1CFD9FFE652DF6ADFCF00F05B0EE76E4F
:100C40000018E8AE02D0E73402D0E750005C12E2B0
:100C5000FE0EDBCFE6FFDFCFE6FFD2DFE552E55247
:100C6000E66A200EE66E98D8E552E552060EDF24BD
:100C7000DF6EE2D7FE0EDBCFE6FFE66AC1DFE552AC
:100C8000E552E552E552E7CFD9FF1200D9CFE6FF92
:100C9000E1CFD9FF020EE126E66AE66AB1DFE5524E
:100CA000E552DE6ADD6ADECF00F0DDCF01F0D890DC
:100CB000015004E6600E005C000E015825E2E66A71
:100CC0005DDFE552E66A5ADFE552E66A57DFE55234
:100CD000E66A54DFE552E66A51DFE552E66A4EDF26
:100CE000E552E66A4BDFE552E66A48DFE552DECFC1
:100CF00000F0DDCF01F0080E0026000E012200C03A
:100D0000DEFF01C0DDFFCFD7E66AE66A79DFE55294
:100D1000E552020EE15C02E2E16AE552E16EE55263
:100D2000E7CFD9FF1200D9CFE6FFE1CFD9FFE652D6
:100D3000DF6ADFCF00F0080EE76E0018E8AE02D0E1
:100D4000E73402D0E750005C22E2DFCFE6FFFE0E80
:100D5000DBCFE6FF55DFE552E552E66A0FDFE552ED
:100D6000E66A0CDFE552E66A09DFE552E66A06DF6D
:100D7000E552E66A03DFE552E66A00DFE552E66A1D
:100D8000FDDEE552E66AFADEE552DF2AD2D7E55209
:100D9000E552E7CFD9FF1200D9CFE6FFE1CFD9FF67
:100DA000FE0EDBCF3FF1200E01013F5D01E246D098
:100DB0003F517F0801E242D0406B050E405D3BE2AF
:100DC000500E3F5D10E2200E3F5D050DF3CF41F167
:100DD00041514025F76A180FF66E4C0EF7220800B5
:100DE000F5CF42F10FD0500E3F5D050DF3CF41F12D
:100DF00041514025F76A080FF66E4D0EF7220800A4
:100E0000F5CF42F142C1E6FFB9DEE552FD0EDBCF80
:100E100000F0000EE76E0018E8AE02D0003403D0F8
:100E2000E750D880005404E242C1E6FFA7DEE55255
:100E30000101402BC2D7E66AA1DEE552E552E7CFB9
:100E4000D9FF1200D9CFE6FFE1CFD9FFE652010169
:100E5000446B456B466B476BDF6AFD0EDB50DF5C16
:100E600007E0D8904437453746374737DF2AF5D76C
:100E7000448344C148F145C149F146C14AF147C1E3
:100E80004BF1496B4A6B4B6B080E1F0B44C14CF185
:100E900045C14DF146C14EF147C14FF108E0010196
:100EA000D8904F334E334D334C33E806F9E101010E
:100EB0004D6B4E6B4F6B100E1F0B44C150F145C173
:100EC00051F146C152F147C153F108E00101D890F8
:100ED0005333523351335033E806F9E10101516B7A
:100EE000526B536B180E1F0B44C154F145C155F1A1
:100EF00046C156F147C157F108E00101D890573378
:100F0000563355335433E806F9E10101556B566BFE
:100F1000576B010EE66EFE0EDBCFE6FF71DEE5528B
:100F2000E55254C1E6FF2AD8E552020EE66EFE0EE7
:100F3000DBCFE6FF65DEE552E55250C1E6FF1ED885
:100F4000E552030EE66EFE0EDBCFE6FF59DEE552FC
:100F5000E5524CC1E6FF12D8E552040EE66EFE0ED5
:100F6000DBCFE6FF4DDEE552E55248C1E6FF06D88D
:100F7000E552E552E552E7CFD9FF1200D9CFE6FF9F
:100F8000E1CFD9FFE65282828290080EDF6EDFCF7A
:100F900000F0000EE76E0018E8AE02D0003403D077
:100FA000E750D880005415E282960A0EE66E97EC60
:100FB00001F0E552FE0EDBB002D0829801D08288AB
:100FC0008286DB407F0BE76EFE0EE7CFDBFFDF069E
:100FD000DED78280E552E552E7CFD9FF1200E66AFC
:100FE00025DEE552010EE66E21DEE552020EE66ECA
:100FF0001DDEE552030EE66E19DEE552040EE66EC6
:1010000015DEE552050EE66E11DEE552060EE66EC1
:101010000DDEE552070EE66E09DEE5521200D9CF6D
:10102000E6FFE1CFD9FFFD0EDBCFE6FFFE0EDBCF03
:10103000E6FFE6DDE552E552E66A200EE66EACDE3E
:10104000E552E552E552E7CFD9FF1200E66A96DD98
:10105000E552040EE66E92DDE552020EE66E8EDD7E
:10106000E5527F0EE66E8ADDE552020EE66E86DD03
:10107000E552040EE66E82DDE552E66A7FDDE5525A
:10108000E66A7CDDE5521200100EE66E77DDE55271
:10109000200EE66E73DDE5527F0EE66E6FDDE552E3
:1010A000200EE66E6BDDE552100EE66E67DDE55252
:1010B000E66A64DDE552E66A61DDE552E66A5EDD18
:1010C000E5521200080EE66E59DDE5521C0EE66E82
:1010D00055DDE5522A0EE66E51DDE552080EE66E4C
:1010E0004DDDE552080EE66E49DDE552F80EE66E7E
:1010F00045DDE552E66A42DDE552E66A3FDDE5524E
:101100001200080EE66E3ADDE552080EE66E36DD98
:10111000E5522A0EE66E32DDE5521C0EE66E2EDD3D
:10112000E552080EE66E2ADDE552E66A27DDE55255
:10113000E66A24DDE552E66A21DDE5521200E66A40
:101140001DDDE552060EE66E19DDE552090EE66E6E
:1011500015DDE552090EE66E11DDE552060EE66E6E
:101160000DDDE552E66A0ADDE552E66A07DDE55285
:10117000E66A04DDE5521200E66A00DDE552060E7D
:10118000E66EFCDCE5520F0EE66EF8DCE5520F0E63
:10119000E66EF4DCE552060EE66EF0DCE552E66A39
:1011A000EDDCE552E66AEADCE552E66AE7DCE552A8
:1011B0001200D9CFE6FFE1CFD9FFFD0EDBCFE9FF6B
:1011C000FE0EDBCFEAFFEF5012E0FC0EDBCFE6FFB6
:1011D000FD0EDBCFE9FFDB2AFE0EDBCFEAFF01E3EA
:1011E000DB2AEF50E66ED8DDE552E552E6D7E55250
:1011F000E7CFD9FF1200D9CFE6FFE1CFD9FF020E2A
:10120000E1260A0EDE6EDD6A000EDFCF20F0010E51
:10121000DBCF21F049EC20F01FC035F120C036F1C2
:1012200021C037F122C038F1770E006ECC0E016E6E
:10123000AB0E026E420E036E35C124F036C125F0AE
:1012400037C126F038C127F000C01FF001C020F0E0
:1012500002C021F003C022F063EC21F01FC031F185
:1012600020C032F121C033F122C034F131C1E6FF98
:1012700032C1E6FF33C1E6FF34C1E6FFDBEC2BF001
:10128000E552E552E552E5521EC000F01FC001F0E4
:1012900020C002F021C003F000C01FF001C020F008
:1012A00002C021F003C022F04AEC22F01EC085F2F9
:1012B0001FC086F220C087F221C088F2000EE66EC1
:1012C000E66A85C2E6FF86C2E6FF87C2E6FF88C2FD
:1012D000E6FFC5DA006E060EE15E0050010EE66E16
:1012E000000EE66E020EE66E31C1E6FF32C1E6FF89
:1012F00033C1E6FF34C1E6FF1DEC0EF0006E070EB1
:10130000E15E0050000EE66E020EE66E5CEC01F04F
:10131000E552E552F3CF17F1F4CF18F1090EE66E5E
:10132000F5EC00F0E552060EE66E80DCE552E66A6A
:10133000000EE66E020EE66E3CDFE552E552E55227
:10134000050EE66E73DCE552DECFE6FFDDCFE6FF8D
:10135000130E006E000E016E026A00C0E6FF01C0AF
:10136000E6FF02C0E6FF000EE66E020EE66E63ECDC
:101370002CF0036E070EE15E0350E66A000EE66E87
:10138000020EE66E16DFE552E552E552000EE66EFD
:10139000020EE66E5CEC01F0E552E552F3CF17F178
:1013A000F4CF18F1090EE66EF5EC00F0E552DECF51
:1013B00000F0DDCF01F0050E0026000E012200C076
:1013C000DEFF01C0DDFFD9CFE9FFDACFEAFF640E0F
:1013D000D880EE54000EED540CE2DECF00F0DDCFED
:1013E00001F00F0E0026000E012200C0DEFF01C03A
:1013F000DDFFD9CFE9FFDACFEAFFE80ED880EE545F
:10140000030EED540CE2DECF00F0DDCF01F01E0E36
:101410000026000E012200C0DEFF01C0DDFFD9CF93
:10142000E9FFDACFEAFF100ED880EE54270EED5414
:101430000CE2DECF00F0DDCF01F0320E0026000E10
:10144000012200C0DEFF01C0DDFF8EEC01F0880E3E
:10145000E66E130EE66EE66AE66AEBEC12F0E55213
:10146000E552E552E552D9CFE9FFDACFEAFF200E87
:10147000D880EE544E0EED5401E3C6D6020EE15C68
:1014800002E2E16AE552E16EE552E7CFD9FF1200D0
:10149000060EE66E16EC06F0E552A0C120F0A1C1E2
:1014A00021F04BEC20F01FC000F020C001F021C063
:1014B00002F022C003F000C024F001C025F002C0F9
:1014C00026F003C027F035C11FF036C120F037C128
:1014D00021F038C122F07AEC20F01FC039F120C091
:1014E0003AF121C03BF122C03CF1770E006ECC0EE8
:1014F000016EAB0E026E420E036E39C124F03AC18A
:1015000025F03BC126F03CC127F000C01FF001C010
:1015100020F002C021F003C022F063EC21F01FC0D4
:1015200031F120C032F121C033F122C034F131C198
:10153000E6FF32C1E6FF33C1E6FF34C1E6FFDBEC74
:101540002BF0E552E552E552E5521EC000F01FC0F7
:1015500001F020C002F021C003F000C01FF001C064
:1015600020F002C021F003C022F04AEC22F01EC09D
:1015700021F11FC022F120C023F121C024F121C19B
:10158000E6FF22C1E6FF23C1E6FF24C1E6FF0E0EFF
:10159000006E000E016E026A00C0E6FF01C0E6FFA9
:1015A00002C0E6FF000EE66E020EE66E63EC2CF063
:1015B000036E090EE15E0350000EE66EE66A21C17D
:1015C000E6FF22C1E6FF23C1E6FF24C1E6FF47D9BB
:1015D000006E060EE15E0050E66A000EE66E020E38
:1015E000E66EE7DDE552E552E552050EE66E16ECD5
:1015F00006F0E55239C1E6FF3AC1E6FF3BC1E6FF1E
:101600003CC1E6FFDBEC2BF0E552E552E552E5523A
:101610001EC000F01FC001F020C002F021C003F086
:1016200000C01FF001C020F002C021F003C022F072
:101630004AEC22F01EC021F11FC022F120C023F18C
:1016400021C024F121C1E6FF22C1E6FF23C1E6FF4C
:1016500024C1E6FF0E0E006E000E016E026A00C08D
:10166000E6FF01C0E6FF02C0E6FF000EE66E020ED6
:10167000E66E63EC2CF0036E090EE15E0350010E82
:10168000E66E000EE66E020EE66E93DDE552E55262
:10169000E552090EE66EF5EC00F0E552000EE66E3E
:1016A000020EE66E5CEC01F0E552E552F3CF17F165
:1016B000F4CF18F11200D9CFE6FFE1CFD9FF040E25
:1016C000E126DE6ADD6ADECF00F0DDCF01F0D890E2
:1016D000015004E6110E005C000E01586AE2DECFF4
:1016E000E9FFDDCFEAFFB30EE926020EEA22EF5052
:1016F0000101A65D59E1DECFE9FFDDCFEAFFC50EAE
:10170000E926020EEA22EFCF00F0016A00BE01686E
:10171000020E00C0DBFF030E01C0DBFF020EDBCFB9
:10172000E9FF030EDBCFEAFFD890E936EA368D0EEB
:10173000E926020EEA22EECF00F0EFCF01F0026AB6
:1017400000C0E6FF01C0E6FF02C0E6FF000EE66E45
:10175000020EE66E08EC2DF0036E050EE15E0350FE
:10176000000EE66E020EE66E5CEC01F0E552E5520C
:10177000020EF3CFDBFF030EF4CFDBFF090EE66EA4
:10178000F5EC00F0E552030EE66E310EE66E00EC6D
:1017900006F0E552E552E66A000EE66E020EE66ECF
:1017A00008DDE552E552E552DF2A010E01E3DB2AAE
:1017B0008AD7040EE15C02E2E16AE552E16EE5528D
:1017C000E7CFD9FF1200D9CFE6FFE1CFD9FF020E54
:1017D000E126829A100EDE6EDD6ADECF00F0DDCFEC
:1017E00001F0013404E200500008000E01542CE224
:1017F000FE0EDB50800B02E1829801D082880A0E37
:10180000E66E97EC01F0E55282860A0EE66E97ECE2
:1018100001F0E55282960A0EE66E97EC01F0E55271
:10182000FD0EDBCF00F0FE0EDBCF01F0D8900036CE
:101830000136FD0E00C0DBFFFE0E01C0DBFFDF0640
:10184000010E01E2DB06C9D7828A020EE15C02E2E8
:10185000E16AE552E16EE552E7CFD9FF1200D9CF38
:10186000E6FFE1CFD9FFFB0EDBCF2DF1FC0EDBCF86
:101870002EF1FD0EDBCF2FF1FE0EDBCF30F1D95074
:10188000F90FE96EFF0EDA20EA6E000ED880EE54F2
:10189000000EED5439E201012D51016A000F006E76
:1018A000340E012200C0E6FF01C0E6FF8CDFE552E6
:1018B000E55201012E51016A000F006E250E012232
:1018C00000C0E6FF01C0E6FF7EDFE552E552010100
:1018D0002F51016A000F006E360E012200C0E6FF94
:1018E00001C0E6FF70DFE552E55201013051016AA7
:1018F000000F006E270E012200C0E6FF01C0E6FFC8
:1019000062DFE552E55238D001012D51016A000F26
:10191000006E300E012200C0E6FF01C0E6FF53DF7B
:10192000E552E55201012E51016A000F006E210EB1
:10193000012200C0E6FF01C0E6FF45DFE552E552A7
:1019400001012F51016A000F006E320E012200C00A
:10195000E6FF01C0E6FF37DFE552E55201013051F5
:10196000016A000F006E230E012200C0E6FF01C0D5
:10197000E6FF29DFE552E552E552E7CFD9FF120035
:10198000000EE66E020EE66E2DC1E6FF2EC1E6FFEA
:101990002FC1E6FF30C1E6FF4FEC25F0006E060ECA
:1019A000E15E0050000EE66E020EE66E5CEC01F0A9
:1019B000E552E552F3CF17F1F4CF18F1090EE66EB8
:1019C000F5EC00F0E55230C1E6FFA9EC12F0E5526B
:1019D000090EE66EF5EC00F0E5522FC1E6FFA9EC2A
:1019E00012F0E552090EE66EF5EC00F0E5522EC15C
:1019F000E6FFA9EC12F0E552090EE66EF5EC00F0F8
:101A0000E5522DC1E6FFA9EC12F0E552090EE66E93
:101A1000F5EC00F0E5528EEF01F0D9CFE6FFE1CF13
:101A2000D9FF0A0EE12601014B0E006F020E016F75
:101A3000FC0EDBCF00F0010EE76E0018E8AE02D01E
:101A4000003403D0E750D880005401E2ECD0FC0E03
:101A5000DB5028E1FD0EDBCF00F0FE0EDBCF01F006
:101A6000060E00C0DBFF070E01C0DBFF080EDB6ABD
:101A7000090EDB6A4B0EE66E020EE66ED950060FBB
:101A8000E96EDACFEAFFEECFE6FFEECFE6FFEECF6C
:101A9000E6FFEFCFE6FF4FEC25F0006E060EE15EAD
:101AA000005010D04B0EE66E020EE66EFD0EDBCF40
:101AB000E6FFFE0EDBCFE6FFB5EC24F0E552E55283
:101AC000E552E55201010AAD84D04B0EE66E020EDE
:101AD000E66E21EC2DF0E552E552020EF3CFDBFF6E
:101AE000030EF4CFDBFFDE6ADD6ADECF00F0DDCF70
:101AF00001F0020EDBCF02F0030EDBCF03F0025049
:101B0000005C035001582EE2020EDBCF02F0030E00
:101B1000DBCF03F0DE50025CE96EDD500358EA6E65
:101B2000E906000EEA5A4B0EE926020EEA22EF50B1
:101B3000E66EFC0EDB50040F006E016A00BE016809
:101B4000DE50005CE96EDD500158EA6E4B0EE9266E
:101B5000020EEA22E552E750EF6EDF2A010E01E3A2
:101B6000DB2AC3D7DE6ADD6ADECF00F0DDCF01F00D
:101B7000FC0EDB50050F046E056A04BE0568020EFC
:101B8000DB50045C026E030EDB500558036E0250FE
:101B9000005C035001581DE201010AA90BD0DECF01
:101BA000E9FFDDCFEAFF4B0EE926020EEA22300EF6
:101BB000EF6E0AD0DECFE9FFDDCFEAFF4B0EE9265C
:101BC000020EEA22200EEF6EDF2A010E01E3DB2A6D
:101BD000CBD7FC0EDB50050FE96EEA6AE9BEEA6876
:101BE0004B0EE926020EEA22EF6A01010AAF0DD080
:101BF000FB0EDBCFE6FF00C1E6FF01C1E6FFD9EC3B
:101C000008F0E552E552E5520ED000C1E6FF01C1F1
:101C1000E6FF5CEC01F0E552E552020EF3CFDBFF8C
:101C2000030EF4CFDBFF0A0EE15C02E2E16AE5524B
:101C3000E16EE552E7CFD9FF1200D9CFE6FFE1CF41
:101C4000D9FF0E0EE126F90EDBCFDEFFDBCFDDFF85
:101C5000F80EDBCF02F0000EE76E0218E8AE02D0FD
:101C6000023403D0E750D880025402E3070E12D0AA
:101C7000F80EDBCF03F0160EE76E0318E8AE02D0C5
:101C8000033403D0E750D880035402E2170E02D089
:101C9000F80EDB28006E016A00BE0168080E00C065
:101CA000DBFF090E01C0DBFF020EDB6A030EDB6AFD
:101CB000FB0EDBCF00F0FC0EDBCF01F0FD0EDBCF27
:101CC00002F0FE0EDBCF03F0246A256A266A276A3B
:101CD00000C01FF001C020F002C021F003C022F0BC
:101CE0008AEC22F0010A33E1F90EDBCFE9FFDB2AAF
:101CF000FA0EDBCFEAFF01E3DB2A2D0EEF6EFB0EBF
:101D0000DBCF00F0FC0EDBCF01F0FD0EDBCF02F0ED
:101D1000FE0EDBCF03F0246A256A800E266EBF0E0E
:101D2000276E00C01FF001C020F002C021F003C0E8
:101D300022F063EC21F0FB0E1FC0DBFFFC0E20C085
:101D4000DBFFFD0E21C0DBFFFE0E22C0DBFFFB0E22
:101D5000DBCF00F0FC0EDBCF01F0FD0EDBCF02F09D
:101D6000FE0EDBCF03F0246A256A266A276A00C0CC
:101D70001FF001C020F002C021F003C022F081EC6E
:101D800022F0010A4AE1FB0EDBCF00F0FC0EDBCFB4
:101D900001F0FD0EDBCF02F0FE0EDBCF03F0246A74
:101DA000256A800E266E3F0E276E00C01FF001C010
:101DB00020F002C021F003C022F08AEC22F0010AD8
:101DC0002CE1006A016A200E026E410E036ED950AA
:101DD000FB0FE96EFF0EDA20EA6EEECF1FF0EECFBA
:101DE00020F0EECF21F0EFCF22F000C024F001C0B0
:101DF00025F002C026F003C027F063EC21F022C0DA
:101E0000EDFF21C0EDFF20C0EDFF1FC0EFFF020E70
:101E1000DB06030E01E2DB06B6D7FB0EDBCF00F0DC
:101E2000FC0EDBCF01F0FD0EDBCF02F0FE0EDBCFB0
:101E300003F0246A256A200E266E410E276E00C02C
:101E40001FF001C020F002C021F003C022F08AEC94
:101E500022F0010A2EE0FB0EDBCF00F0FC0EDBCF00
:101E600001F0FD0EDBCF02F0FE0EDBCF03F0246AA3
:101E7000256A200E266E410E276E00C01FF001C09D
:101E800020F002C021F003C022F010EC21F0FB0E84
:101E90001FC0DBFFFC0E20C0DBFFFD0E21C0DBFFFF
:101EA000FE0E22C0DBFF020EDB2A030E01E3DB2A5B
:101EB000B4D7020EDBCF00F0030EDBCF01F0D95018
:101EC000080FE96EDACFEAFF0050EE260150ED224E
:101ED000010EF36E040EF3CFDBFF050EDB6A040E7A
:101EE000DBCF20F0050EDBCF21F04BEC20F00A0E0B
:101EF0001FC0DBFF0B0E20C0DBFF0C0E21C0DBFF81
:101F00000D0E22C0DBFF040EDBCF00F0050EDBCF91
:101F100001F0080EDBCF02F0090EDBCF03F0015019
:101F20000318E8AE02D0033404D00250005C035022
:101F300001582EE20A0EDBCF00F00B0EDBCF01F0D2
:101F40000C0EDBCF02F00D0EDBCF03F0246A256A06
:101F5000200E266E410E276E00C01FF001C020F03B
:101F600002C021F003C022F010EC21F00A0E1FC0C5
:101F7000DBFF0B0E20C0DBFF0C0E21C0DBFF0D0EC4
:101F800022C0DBFF040EDB2A050E01E3DB2ABBD7F0
:101F90000A0EDBCF04F00B0EDBCF05F00C0EDBCF0F
:101FA00006F00D0EDBCF07F0246A256A266A400E84
:101FB000276E04C01FF005C020F006C021F007C046
:101FC00022F010EC21F01FC000F020C001F021C071
:101FD00002F022C003F0D950FB0FE96EFF0EDA20A9
:101FE000EA6EEECF1FF0EECF20F0EECF21F0EFCF74
:101FF00022F000C024F001C025F002C026F003C08A
:1020000027F07AEC20F022C0EDFF21C0EDFF20C0C8
:10201000EDFF1FC0EFFFFB0EDBCF00F0FC0EDBCFB0
:1020200001F0FD0EDBCF02F0FE0EDBCF03F0246AE1
:10203000256A200E266E410E276E00C01FF001C0DB
:1020400020F002C021F003C022F08AEC22F0010A45
:1020500013E0FB0EDB6AFC0EDB6A800EF36EFD0EF6
:10206000F3CFDBFF3F0EF36EFE0EF3CFDBFF020E6E
:10207000DB2A030E01E3DB2A020EDBCF00F0030EA6
:10208000DBCF01F00001800E01145FE0F90EDBCF21
:10209000E9FFDB2AFA0EDBCFEAFF01E3DB2A300E91
:1020A000EF6EF90EDBCFE9FFDB2AFA0EDBCFEAFF9A
:1020B00001E3DB2A2E0EEF6E080EDBCF00F0090ED7
:1020C000DBCF01F0800E011414E0020EDBCF02F032
:1020D000030EDBCF03F0080EDB50025C006E090E2E
:1020E000DB500358016E020E00C0DBFF030E01C07F
:1020F000DBFF040EDB68050EDB68040EDBCF00F0AF
:10210000050EDBCF01F0020EDBCF02F0030EDBCFBA
:1021100003F003500118E8AE02D0013404D000509F
:10212000025C0150035811E2F90EDBCFE9FFDB2A14
:10213000FA0EDBCFEAFF01E3DB2A300EEF6E040E6E
:10214000DB06050E01E2DB06D8D7040EDB6A050EBE
:10215000DB6A040EDBCF00F0050EDBCF01F0080ECA
:10216000DBCF02F0090EDBCF03F001500318E8AE1D
:1021700002D0033404D00250005C0350015801E344
:10218000ACD0FB0EDBCF1FF0FC0EDBCF20F0FD0E42
:10219000DBCF21F0FE0EDBCF22F01BEC22F0060E8F
:1021A00020C0DBFF070E21C0DBFF300EE76E060EFE
:1021B000DBCF00F0070EDBCF01F0E7500026000E6A
:1021C0000122F90EDBCFE9FFDB2AFA0EDBCFEAFFB3
:1021D00001E3DB2A00C0EFFF040EDBCF00F0050EA9
:1021E000DBCF01F0020EDB50001803E1030EDB50E1
:1021F00001180BE1F90EDBCFE9FFDB2AFA0EDBCF8A
:10220000EAFF01E3DB2A2E0EEF6E060EDBCF20F095
:10221000070EDBCF21F04BEC20F00A0E1FC0DBFFD6
:102220000B0E20C0DBFF0C0E21C0DBFF0D0E22C009
:10223000DBFF1FC000F020C001F021C002F022C06F
:1022400003F0D950FB0FE96EFF0EDA20EA6EEECFF5
:102250001FF0EECF20F0EECF21F0EFCF22F000C044
:1022600024F001C025F002C026F003C027F079EC6D
:1022700020F022C0EDFF21C0EDFF20C0EDFF1FC008
:10228000EFFF006A016A200E026E410E036ED95004
:10229000FB0FE96EFF0EDA20EA6EEECF1FF0EECFF5
:1022A00020F0EECF21F0EFCF22F000C024F001C0EB
:1022B00025F002C026F003C027F063EC21F022C015
:1022C000EDFF21C0EDFF20C0EDFF1FC0EFFF040EAA
:1022D000DB2A050E01E3DB2A3CD7F90EDBCFE9FF51
:1022E000FA0EDBCFEAFFEF6A0E0EE15C02E2E16A72
:1022F000E552E16EE552E7CFD9FF1200D9CFE6FFF4
:10230000E1CFD9FF060EE12601010A9DFB0EDBCFCE
:102310001FF0FC0EDBCF20F0FD0EDBCF21F0FE0E18
:10232000DBCF22F04AEC22F01EC0DEFF1FC0DEFF32
:1023300020C0DEFF21C0DDFFDD52DD52FB0EDBCF12
:1023400004F0FC0EDBCF05F0FD0EDBCF06F0FE0E39
:10235000DBCF07F0F90EDBCF20F0FA0EDBCF21F058
:102360004BEC20F01FC008F020C009F021C00AF09B
:1023700022C00BF008C024F009C025F00AC026F0E6
:102380000BC027F004C01FF005C020F006C021F0EC
:1023900007C022F063EC21F01FC000F020C001F064
:1023A00021C002F022C003F0F90EDBCF14F0FA0EC8
:1023B000DBCF15F0166A176A15AE02D016681768DB
:1023C00014C01EF015C01FF016C020F017C021F079
:1023D000DFCF23F0010EDBCF24F0020EDBCF25F0A0
:1023E000030EDBCF26F096EC2DF01AC010F01BC0C8
:1023F00011F01CC012F01DC013F010C01EF011C06F
:102400001FF012C020F013C021F060EC20F01FC0BC
:102410000CF020C00DF021C00EF022C00FF00CC057
:1024200024F00DC025F00EC026F00FC027F000C02C
:102430001FF001C020F002C021F003C022F079ECAF
:1024400020F01BEC22F0040E20C0DBFF050E21C0A3
:10245000DBFF000EE66E020EE66ED9CFE9FFDACFA3
:10246000EAFFEECFE6FFEECFE6FFEECFE6FFEFCFDF
:10247000E6FF4FEC25F0006E060EE15E0050010114
:102480000AAF0DD0F80EDBCFE6FF000EE66E020EAF
:10249000E66ED9EC08F0E552E552E5520CD0000E9C
:1024A000E66E020EE66E5CEC01F0E552E552F3CF0B
:1024B00017F1F4CF18F101010AAF0AD0F80EDBCF03
:1024C000E6FF2E0EE66ECCEC06F0E552E55205D0A6
:1024D0002E0EE66EF5EC00F0E552F80EDBCFE6FFCF
:1024E000E66A040EDBCFE6FF050EDBCFE6FF0DEC60
:1024F0000DF0E552E552E552E552060EE15C02E2CE
:10250000E16AE552E16EE552E7CFD9FF1200D9CF7B
:10251000E6FFE1CFD9FFE652800EDF6EDF50000804
:1025200013E2FE0EDB50DF1406E0310EE66EF5EC32
:1025300000F0E55205D0300EE66EF5EC00F0E55205
:10254000DF407F0BDF6EEAD7E552E552E7CFD9FFD8
:102550001200D9CFE6FFE1CFD9FF020EE126FE0E31
:10256000DB50F00BE8380F0B300FDF6EDF5039080F
:1025700003E2070EDF24DF6EFE0EDB500F0B300F81
:10258000E76E010EE7CFDBFFDB5039080AE2070EEA
:10259000006E010EDBCFE7FF0050E726010EE7CF0C
:1025A000DBFFDFCFE6FFF5EC00F0E552010EDBCFFD
:1025B000E6FFF5EC00F0E552680EE66EF5EC00F093
:1025C000E552020EE15C02E2E16AE552E16EE5529B
:1025D000E7CFD9FF1200D9CFE6FFE1CFD9FFFB0E3D
:1025E000DBCF1FF0FC0EDBCF20F0FD0EDBCF21F0A8
:1025F000FE0EDBCF22F02234000E221809E6D8802E
:10260000000E1F54000E2054000E2154000E2254C0
:102610000CE2D950FB0FE96EFF0EDA20EA6EEE06EF
:10262000000EEE5AEE5AEE5ADAD7E552E7CFD9FF4E
:102630001200D9CFE6FFE1CFD9FF020EE126DE6A14
:10264000DD6ADECF00F0DDCF01F0FE0EDB500001D1
:1026500001AE02D0D89003D0005C000E01580AE20F
:10266000200EE66EF5EC00F0E552DF2A010E01E3E4
:10267000DB2AE7D7020EE15C02E2E16AE552E16E95
:10268000E552E7CFD9FF12006F6A6E6A8168FD0ECE
:10269000936E93809392938493869388938A938C7A
:1026A000938EC26A070EC16E926E896A8268800E2E
:1026B000946E94909492949494969498949A949CF2
:1026C000948E1200DACFE4FFE2CFDAFFE9CFE4FF25
:1026D000EACFE4FFE652D9CFE6FFE1CFD9FFE652D9
:1026E0009EAA16D0AE50DF6E010104C1E9FF05C1FC
:1026F000EAFF042B000E0523DFCFEFFF830E045DFE
:10270000020E055904E35B0E046F020E056F9E9ADC
:10271000E552E552E7CFD9FFE552E5CFEAFFE5CF35
:10272000E9FFE5CFDAFF1100DACFE4FFE2CFDAFF0D
:10273000E9CFE4FFEACFE4FFF3CFE4FFF4CFE4FF17
:10274000E652D9CFE6FFE1CFD9FF040EE126F2A28F
:10275000A6D0010E2C6EF150400B01E0010E2C5C56
:10276000E8B0F18CE8A0F19C81CF12F1F292D65042
:10277000DE6EDD6AD66A01019851020A60E0030A42
:102780000DE0010A01E08BD0010E996F9A6B9B6FEF
:102790009D6B9C6F986FF294F28A81D0D9CFE9FF3C
:1027A000DACFEAFF230ED880EE54000EED5443E258
:1027B000DECF2CF0DDCF2DF0B00E2C5C000E2D58AE
:1027C0003AE2DECF2CF0DDCF2DF0680E2C5C000E4F
:1027D0002D5815E29D2B020E9D5D10E1010ED89043
:1027E00099379A37E806FBE101019C512C6E2D6A5E
:1027F0002C5099132D509A139B2B9D6B14D0010EC6
:10280000D8809C559C6F010ED89099379A37E8066E
:10281000FBE101019C512C6E2D6A2C5099132D5017
:102820009A139B2B9D6B0E0E9B5D04E1020E986F1D
:10283000F19CF29A03D0986BF19CF29A30D0F19C03
:102840009A512D6AE830E830E8301F0B2C6E2C507E
:10285000010B02E0000E01D0010E9E91E8B09E81B6
:1028600099C12CF09AC12DF0060ED8902D322C3241
:10287000E804FBE11F0E2C1401011F0BF36EF3465D
:10288000C10E9E15F3109E6F3F0E99153F0BF36E10
:10289000C00E9F15F3109F6F9F8D986B00D0F2A410
:1028A00007D080780101980503E1986BF19CF29ABA
:1028B000F294040EE15C02E2E16AE552E16EE55257
:1028C000E7CFD9FFE552E5CFF4FFE5CFF3FFE5CF42
:1028D000EAFFE5CFE9FFE5CFDAFF1100980EE66EDB
:1028E0003A0EE66EE66AE66A76DEE552E552E552B3
:1028F000E552CADE01015B0E046F020E056F04C1D2
:1029000002F105C103F1BEEC00F00C0EE66EF5EC31
:1029100000F0E552A00EE66E860EE66E010EE66E43
:10292000E66A59DEE552E552E552E5528EEC01F0D9
:102930000201000E496F020E4A6F01014B0E006F3B
:10294000020E016FDBC200F0DCC201F0026A00C0BF
:10295000E6FF01C0E6FF02C0E6FF49C2E6FF4AC249
:10296000E6FF08EC2DF0036E050EE15E035049C250
:10297000E6FF4AC2E6FF5CEC01F0E552E552F3CF18
:1029800017F1F4CF18F1EFC200F0F0C201F0026AC3
:1029900000C0E6FF01C0E6FF02C0E6FF000EE66EE3
:1029A000020EE66E08EC2DF0036E050EE15E03509C
:1029B000000EE66E020EE66E5CEC01F0E552E552AA
:1029C000F3CF17F1F4CF18F1000EE66EE66A75EC5E
:1029D00000F0E552E552800EE66EE66A75EC00F016
:1029E000E552E552A00EE66EE66A75EC00F0E5529F
:1029F000E552C00EE66EE66A75EC00F0E552E5526F
:102A0000E00EE66EE66A75EC00F0E552E5528EECFB
:102A100001F0200EE66E4E0EE66EE66AE66ADBDD3B
:102A2000E552E552E552E552808680880101986BB7
:102A30000A9F5CEC05F08AEC05F046EC06F0E66ACD
:102A4000E66A00EC06F0E552E552F1C200F0F2C28F
:102A500001F0026A00C0E6FF01C0E6FF02C0E6FF27
:102A6000000EE66E020EE66E08EC2DF0036E050E0B
:102A7000E15E0350E66A000EE66E020EE66ED9ECE9
:102A800008F0E552E552E552E66AD00EE66EE3EC58
:102A90000BF0E552E552010EE66EE66A00EC06F038
:102AA000E552E552F3C200F0F4C201F0026A00C040
:102AB000E6FF01C0E6FF02C0E6FF000EE66E020E72
:102AC000E66E08EC2DF0036E050EE15E0350E66A3B
:102AD000000EE66E020EE66ED9EC08F0E552E55205
:102AE000E552200EE66E4E0EE66EE66AE66A73DD8D
:102AF000E552E552E552E5520101A20E2D6FEE0EB0
:102B00002E6F030E2F6F306BA20EE66E300EE66E48
:102B1000E3EC0BF0E552E552EE0EE66E210EE66EAA
:102B2000E3EC0BF0E552E552030EE66E320EE66E74
:102B3000E3EC0BF0E552E552E66A230EE66EE3ECB9
:102B40000BF0E552E552020EE66EE66A00EC06F086
:102B5000E552E552F5C200F0F6C201F0026A00C08B
:102B6000E6FF01C0E6FF02C0E6FF000EE66E020EC1
:102B7000E66E08EC2DF0036E050EE15E0350E66A8A
:102B8000000EE66E020EE66ED9EC08F0E552E55254
:102B9000E552E66A900EE66EE3EC0BF0E552E55284
:102BA000E66AC00EE66EE3EC0BF0E552E552A80EC5
:102BB000E66E610EE66EE66AE66A0DDDE552E55206
:102BC000E552E552E66A500EE66EE3EC0BF0E55294
:102BD000E552040EE66EE66A00EC06F0E552E552B8
:102BE000F9C200F0FAC201F0026A00C0E6FF01C0BB
:102BF000E6FF02C0E6FF000EE66E020EE66E08EC8F
:102C00002DF0036E050EE15E0350E66A000EE66EDF
:102C1000020EE66ED9EC08F0E552E552E552A00E40
:102C2000E66E860EE66E010EE66EE66AD4DCE552CE
:102C3000E552E552E552640E01011B6F1C6B0F6BF0
:102C4000106B216B226B236B246B256B266B276B20
:102C5000286B0A9DDFC200F0E0C201F0026A00C0EA
:102C6000E6FF01C0E6FF02C0E6FF000EE66E020EC0
:102C7000E66E08EC2DF0036E050EE15E0350000ECB
:102C8000E66E020EE66E5CEC01F0E552E552F3CF23
:102C900017F1F4CF18F18EEC01F0EDC200F0EEC2A6
:102CA00001F0026A00C0E6FF01C0E6FF02C0E6FFD5
:102CB000000EE66E020EE66E08EC2DF0036E050EB9
:102CC000E15E0350000EE66E020EE66E5CEC01F073
:102CD000E552E552F3CF17F1F4CF18F1100EE66E7E
:102CE000270EE66EE66AE66A76DCE552E552E552C4
:102CF000E55201019F9D020EAA6FA06BA16B066BAE
:102D0000076B540EE66E17EC2EF0E552FC0EE66EE5
:102D1000CEEC2DF0E552F26AF16AF184F180D08EAA
:102D2000D66AD58EF28CF28AF28EF292F288010186
:102D30009FAD90D3F29880969E513E0BE842A46FCF
:102D4000A56B9F513F0BA66FA76B9F9D9E51010BDB
:102D5000AA5D04E1A82B000EA92305D0A86BA96BDE
:102D60009E51010BAA6F030EE66E16EC06F0E552BB
:102D70008DC200F08EC201F0026A00C0E6FF01C001
:102D8000E6FF02C0E6FF000EE66E020EE66E08ECFD
:102D90002DF0036E050EE15E0350000EE66E020E8E
:102DA000E66E5CEC01F0E552E552F3CF17F1F4CF9B
:102DB00018F1E66A000EE66E020EE66ED9EC08F037
:102DC000E552E552E552E66AE66AA6C1E6FFA7C10A
:102DD000E6FF0DEC0DF0E552E552E552E552200E0E
:102DE000E66EF5EC00F0E552090EE66EF5EC00F04B
:102DF000E552020EE66E16EC06F0E552FBC200F05C
:102E0000FCC201F0026A00C0E6FF01C0E6FF02C09A
:102E1000E6FF000EE66E020EE66E08EC2DF0036E85
:102E2000050EE15E0350E66A000EE66E020EE66EE7
:102E3000D9EC08F0E552E552E552E66A200EE66E5E
:102E4000CCEC06F0E552E552030EE66E1C0EE66E83
:102E500000EC06F0E552E552E66A00C1E6FF01C16A
:102E6000E6FFD9EC08F0E552E552E5525BEC0BF0D9
:102E70003C0E0101A61901E1A75101E1E0D2310E9A
:102E8000A61901E1A75101E1C4D22E0EA61901E154
:102E9000A75101E1BDD22C0EA61901E1A75101E114
:102EA000B6D22B0EA61901E1A75101E1AFD2290E2E
:102EB000A61901E1A75101E16CD2260EA61901E184
:102EC000A75101E165D2220EA61901E1A75101E146
:102ED00032D21D0EA61901E1A75101E12BD21C0E21
:102EE000A61901E1A75101E124D2190EA61901E1A9
:102EF000A75101E11DD2180EA61901E1A75101E168
:102F000016D2170EA61901E1A75101E132D1110E17
:102F1000A61901E1A75101E11AD1100EA61901E18C
:102F2000A75101E102D10F0EA61901E1A75101E15C
:102F30008ED00D0EA61901E1A75101E187D0A6514F
:102F400001E1A7512EE0010EA61901E1A75129E0E8
:102F5000020EA61901E1A75124E0030EA61901E112
:102F6000A7511FE0040EA61901E1A7511AE0050EB2
:102F7000A61901E1A75115E0060EA61901E1A75116
:102F800010E0070EA61901E1A7510BE0080EA619E3
:102F900001E1A75106E0090EA61901E1A75101E0E0
:102FA0004FD20651071106E10A87050EE66E16ECB0
:102FB00006F0E55201010AA748D0300EA625E66EBC
:102FC000400E0625E96E020E0721EA6EE552E75033
:102FD000EF6E050EE66E0C0E206E216A06C125F01E
:102FE00007C126F0FDEC21F01E50E66E00EC06F065
:102FF000E552E552010EE66E400E01010625E96E2E
:10300000020E0721EA6EEF50E66ECCEC06F0E552B8
:10301000E5520101080E065D000E075903E2062B7A
:10302000000E0723400E0625E96E020E0721EA6E08
:10303000EF6A400EE66E020EE66E5CEC01F0E552C1
:10304000E552F3CF17F1F4CF18F1FAD1F9D1040E0C
:10305000E66E16EC06F0E55201C300F002C301F083
:10306000026A00C0E6FF01C0E6FF02C0E6FF000EF4
:10307000E66E020EE66E08EC2DF0036E050EE15EC4
:103080000350E66A000EE66E020EE66ED9EC08F01A
:10309000E552E552E552F29EFBEC08F0040EE66EB6
:1030A00016EC06F0E552F9C200F0FAC201F0026A2D
:1030B00000C0E6FF01C0E6FF02C0E6FF000EE66EBC
:1030C000020EE66E08EC2DF0036E050EE15E035075
:1030D000E66A000EE66E020EE66ED9EC08F0E552E6
:1030E000E552E552DFC200F0E0C201F0026A00C022
:1030F000E6FF01C0E6FF02C0E6FF000EE66E020E2C
:10310000E66E08EC2DF0036E050EE15E0350000E36
:10311000E66E020EE66E5CEC01F0E552E552F3CF8E
:1031200017F1F4CF18F1F28E8BD1A02B000EA12352
:10313000E66AE66AA0C1E6FFA1C1E6FF0DEC0DF06C
:10314000E552E552E552E55248EC0AF079D1A00784
:10315000000EA15BE66AE66AA0C1E6FFA1C1E6FF38
:103160000DEC0DF0E552E552E552E55248EC0AF05F
:1031700067D1000ED8800655000E075501E3D6D062
:103180000A51080B01E1D2D0400EE66E020EE66E47
:103190000EEC28F0E552E5521EC035F11FC036F1A5
:1031A00020C037F121C038F1770E006ECC0E016ED1
:1031B000AB0E026E420E036E35C124F036C125F00F
:1031C00037C126F038C127F000C01FF001C020F041
:1031D00002C021F003C022F063EC21F01FC031F1E6
:1031E00020C032F121C033F122C034F131C1E6FFF9
:1031F00032C1E6FF33C1E6FF34C1E6FFDBEC2BF062
:10320000E552E552E552E5521EC000F01FC001F044
:1032100020C002F021C003F000C01FF001C020F068
:1032200002C021F003C022F04AEC22F01EC021F1BE
:103230001FC022F120C023F121C024F1D880000E4C
:1032400001012155000E2255000E2355000E245574
:1032500011E2000EE66EE66A21C1E6FF22C1E6FF3A
:1032600023C1E6FF24C1E6FF2FEC0CF0006E060E32
:10327000E15E0050010EE66E000EE66E020EE66E96
:1032800031C1E6FF32C1E6FF33C1E6FF34C1E6FFDC
:103290001DEC0EF0006E070EE15E0050000EE66EB3
:1032A000020EE66E5CEC01F0E552E552F3CF17F149
:1032B000F4CF18F1090EE66EF5EC00F0E552060EBB
:1032C000E66E16EC06F0E552E66A000EE66E020EB9
:1032D000E66ED9EC08F0E552E552E552050EE66ED1
:1032E00016EC06F0E552010EE66E000EE66E020EDA
:1032F000E66E35C1E6FF36C1E6FF37C1E6FF38C1ED
:10330000E6FF1DEC0EF0006E070EE15E0050010EB0
:10331000E66E000EE66E020EE66ED9EC08F0E5529F
:10332000E552E55201010A97066B076B89D088D0F8
:1033300087D086D085D0000ED8800655000E075560
:1033400026E20607000E075B400E0625E96E020E18
:103350000721EA6EEF6A400EE66E020EE66E5CEC46
:1033600001F0E552E552F3CF17F1F4CF18F1050E55
:10337000E66E16EC06F0E552010EE66E400EE66EC5
:10338000020EE66ED9EC08F0E552E552E55258D04F
:1033900057D0000ED8800655000E075536E20A5168
:1033A000080B33E0400E0625E96E020E0721EA6E97
:1033B0002E0EEF6E080E065D000E075903E2062B77
:1033C000000E0723400E0625E96E020E0721EA6E65
:1033D000EF6A400EE66E020EE66E5CEC01F0E5521E
:1033E000E552F3CF17F1F4CF18F1050EE66E16ECA7
:1033F00006F0E552010EE66E400EE66E020EE66E37
:10340000D9EC08F0E552E552E5521AD019D018D09F
:1034100017D0050EE66E16EC06F0E552060EE66EC7
:1034200016EC06F0E5520101066B076B0A970201E4
:10343000406B0101216B226B236B246B01D000D008
:103440008EEC01F0240EE66E33EC2EF0E552808611
:10345000F292F288100EE66E270EE66EE66AE66AD3
:10346000EBEC12F0E552E552E552E55260D4120061
:1034700074EC1FF0FB0EDBCFF3FFDB06F35000090B
:103480000AE0C2EC1FF0FA0E2DEC20F0F3E1011C73
:10349000F1E1010E01D0000EA3EF1FF074EC1FF05C
:1034A0003B0EE12402E3E168E652E16E010EDB6AC5
:1034B000020EDB6AF90EDBCFF6FFFA0EDBCFF7FF69
:1034C000FB0EDBCFF8FF0800F550DF6EDF5002E1A6
:1034D000C7EF1EF0250EDF5C02E0BAEF1EF0030E10
:1034E000DB6A040EDB6A050EDB6A060EDB6A070E7A
:1034F000DB6ADCEC1EF02D0EDF5C0CE02B0EDF5CDB
:1035000009E0200EDF5C06E0230EDF5C03E0300EF6
:10351000DF5C1AE1DF50300A14E0130A0FE0030AFF
:103520000AE00B0A05E0060AE4E1030EDB80E1D7BE
:10353000030EDB82DED7030EDB84DBD7030EDB86D4
:10354000D8D7030EDB88D5D72A0EDF5C1BE1D8EC79
:103550001EF026EC1FF010E0030EDB8020682168CF
:10356000130EDBCF25F0140EDBCF26F0D0EC21F0CC
:10357000040E1EC0DBFF03D0130E0FEC1FF0DCECBB
:103580001EF00BD0090EDB6A7DEC1FF003E0F1ECBE
:103590001FF0FAD7090E0FEC1FF0030EDBB0DB981B
:1035A0002E0EDF5C1BE1DCEC1EF02A0EDF5C0BE173
:1035B000D8EC1EF026EC1FF003E1130E61EC1FF0B7
:1035C000DCEC1EF00BD0090EDB6A7DEC1FF003E093
:1035D000F1EC1FF0FAD7090E61EC1FF0680EDF5C0A
:1035E00007E1DCEC1EF0680EDF5C1DE1030E18D075
:1035F000740EDF5C17E07A0EDF5C14E0480EDF5CCF
:1036000006E0540EDF5C03E05A0EDF5C02E1020EBE
:1036100007D06C0EDF5C03E06A0EDF5C04E1010E94
:10362000B4EC1FF0C9DBDF506E0A01E17FD31E0A44
:1036300001E192D1200A01E18FD13F0A01E149D194
:103640001A0A01E146D10D0A01E143D1200A01E144
:1036500040D13A0A01E13DD1200A01E13AD1260ADE
:1036600001E135D10D0A01E132D11A0A01E1D9D0C7
:10367000200A4AE0300A1FE0460A0EE0250A01E06F
:1036800083D3D950F90FE96EFF0EDA20EA6E010EEE
:10369000EE5E000EEE5AEE5AC2EC1FF0250EE66EFC
:1036A00095DB03E1011C01E169D3BEEC1FF001E2EF
:1036B0006BD3DB2A69D3080EDB6A040EDB500108EA
:1036C00006E2040EDB0486EC1FF0DB508BDB080EF9
:1036D000DB5009E0030EDB50010B05E172DB01E07A
:1036E0004DD3080EDB6A64DBEFCFDFFF36EC20F052
:1036F00003E1011C01E142D3BEEC1FF001E3DB2A30
:1037000060DB01E141D33AD3070EDB5002080FE141
:1037100002EC20F0030EC9EC1FF00E0EEECFDBFF23
:103720000F0EEECFDBFF100EEECFDBFF20D0F70E3B
:10373000DBCF03F0F80EDBCF04F0020E035E000EC9
:10374000045AF70E03C0DBFFF80E04C0DBFF03C012
:10375000E9FF04C0EAFFB9EC1FF0026A0E0E00C0D8
:10376000DBFF0F0E01C0DBFF100E02C0DBFF0E0EF1
:10377000DBCFE6FF0F0EDBCFE6FF100EDBCFE6FF61
:103780002FEC2DF0E552E552E552130E1FC0DBFF82
:10379000140E20C0DBFF060EDB5005E0130EFDEC1F
:1037A0001FF001E26ADB21EC20F002E2130E37DBAE
:1037B000E4EC1FF006E0040EFDEC1FF002E2050E43
:1037C0002EDB030EDBB005D0FCDA01E0D7D2080E09
:1037D000DB6A090EDB6A0E0EDBCFF6FF0F0EDBCFC6
:1037E000F7FF100EDBCFF8FF0800F550DF6EDF505B
:1037F00014E027EC20F011E236EC20F003E1011C8C
:1038000001E1BCD2BBDB01E3DB2A090EDB2AD95084
:103810000E0FE96E000ECBDBE7D7D3DA01E1B4D2AD
:10382000ADD2C6DA110EEECFDBFF120EEDCFDBFF0D
:10383000110EDBCFE6FF120EDBCFE6FF21EC2DF001
:10384000E552E552130EF3CFDBFF140EF4CFDBFF8E
:10385000060EDB5004E0130ED0DB01E20EDB21ECA0
:1038600020F002E2130EDBDAAFDB05E0040EC5DB6D
:1038700002E2050ED4DA030EDBB005D0A2DA01E0D5
:103880007DD2080EDB6A090EDB6A110EDBCFE9FF81
:10389000120EDBCFEAFFEFCFDFFFDF5014E0D7DB04
:1038A00012E2E4DB03E1011C01E168D267DB01E322
:1038B000DB2A090EDB2A110EDB2ADBCFE9FF120E11
:1038C000E8E3DB2AE6D77DDA01E15ED257D2030EC8
:1038D000DB8E070EDB0410E195DB040E5ADB0A0ECB
:1038E000EECFDBFF0B0EEECFDBFF0C0EEECFDBFFE0
:1038F0000D0EEECFDBFF6CD0070EDB5003082CE182
:10390000030EDBAE0DD0B2DA020E76DAEFCF00F0A6
:10391000016A026A036A00AE39D00168026835D0D4
:10392000F70EDBCF01F0F80EDBCF02F0020E015EE6
:10393000000E025AF70E01C0DBFFF80E02C0DBFFDB
:1039400001C0E9FF02C0EAFFEFCF00F00A0E00C09D
:10395000DBFF0B0EDB6A38D0070EDB50020809E1F3
:10396000030EDBAE04D059DB02AE10D00ED055DB17
:103970000DD0030EDBAE12D079DA020E3DDAF9DAA1
:10398000026A036A01AE02D002680368E2DA0C0E32
:1039900002C0DBFF0D0E03C0DBFF1AD0F70EDBCF3A
:1039A00002F0F80EDBCF03F0020E025E000E035AA7
:1039B000F70E02C0DBFFF80E03C0DBFF02C0E9FF19
:1039C00003C0EAFFD6DAC5DA0C0EDB6A0D0EDB6A3D
:1039D000060EDB5005E1010EF36E050EF3CFDBFFA3
:1039E000150EDB6A160EDB6AD950370F006E000E1B
:1039F000DA20016E390E00C0DBFF3A0E01C0DBFF9A
:103A0000380EDB6A080EDB6A0A0EAEDADF50780A7F
:103A100012E0200A10E0280A0CE0200A0AE03F0A1F
:103A200006E00D0A02E0200A08E1020E05D0080EA9
:103A300003D0080EDF26100E97DA030EDBBE02D08D
:103A4000DB92DB94DB50800B24E08ADAD890030E03
:103A5000EB50000A08E6000EEE5C000EEE58000E79
:103A6000EE58000EEE5815E213DA23682468256834
:103A7000266896EC2DF00A0E1AC0DBFF0B0E1BC059
:103A8000DBFF0C0E1CC0DBFF0D0E1DC0DBFF2D0E7F
:103A900008D0030EDBA202D02B0E03D0DBA408D08B
:103AA000200EF36E170EF3CFDBFF150EDB2A02D0CC
:103AB000170EDB6A050EDB5003E1B7D901E189D0AF
:103AC000100E006E5D0E016E000E026E070EDBCF53
:103AD00003F0046A056A066A03C023F004C024F0F8
:103AE00005C025F006C026F0D3D9F3EC2DF0005028
:103AF0001A24F36E01501B20F46E02501C20F86E45
:103B0000F4CFF7FFF3CFF6FF0800090EF5CFDBFF88
:103B1000580EDF5C0FE1610EF36E090E7BD90AE3EC
:103B2000200E006E090EDBCFE7FF0050E75E090EA6
:103B3000E7CFDBFF070EDBCF00F0016A026A036A02
:103B40000FDA00C023F001C024F002C025F003C04A
:103B500026F0EECF1EF0EECF1FF0EECF20F0EFCF2D
:103B600021F0F3EC2DF021C0EDFF20C0EDFF1FC0D0
:103B7000EDFF1EC0EFFF390EDBCFE9FFDB063A0E8B
:103B8000DBCFEAFF01E2DB06090EDBCFEFFF150E0C
:103B9000DB2A4BD995E1030EDBA61DD06F0EDF5C4F
:103BA00006E1C1D918E3150EDB285BDA14D0780ED4
:103BB000DF5C09E0580EDF5C06E0620EDF5C03E0CC
:103BC000420EDF5C08E1020EF36E160EF3CFDBFF50
:103BD00002D0150EDB6A030EDB50100B0EE0040E54
:103BE000DBCF00F0050EDB50D880005406E2060E55
:103BF000DB5003E1040EDB5034DA95D90AE2050EFE
:103C0000DBCFE7FF150EDB50E75E050EE7CFDBFFEE
:103C100002D0050EDB6A040EDBCF00F0160E45D98C
:103C2000D880005414E2160EDBCFE6FF150EDBCF72
:103C3000E6FF040EDBCFE6FF050EDB50E552E75C46
:103C4000E552D880E754E552D880E7545FD9030E97
:103C5000DB50010B0BE1080EDB5008E0B2D801E0AD
:103C60008DD0080EDB50BED8080EDB6A170EDB5075
:103C700007E088D9170EF1D903E1011C01E17ED0DC
:103C8000160EDB5016E07ED9300EE66E9FD802E1AC
:103C9000011C74E077D9DFCFE6FF54EC2DF0E5523C
:103CA000E552E552F4CF01F00001F31C02E1011CE2
:103CB00065E0050EDBCF00F0160EDB50D880005417
:103CC00009E2050EDBCFE7FF160EDB50E75E050EBF
:103CD000E7CFDBFF300EE66E050ECBD94FE1390E94
:103CE000DB2ADBCFE9FF3A0E01E3DB2ADBCFEAFF79
:103CF000090EEFCFDBFFDB500EE044D9090EADD942
:103D000002E1011C3BE0390EDB2ADBCFE9FF3A0E72
:103D1000EDE3DB2AEBD755D831E1160EDBCFE6FF1A
:103D2000080EC3D8E552E7245DD82ED0070EDB502D
:103D3000030A1CE0010A14E0030A07E07BD9DBCF89
:103D4000EEFF020EDBCFEDFF1FD0F5D8056A03AE04
:103D500002D0046805682CD8BCD805C0EEFF14D08A
:103D6000EAD803BE046824D8B4D80ED063D9DBCF18
:103D7000EFFF0AD07BD905E1011C03E1F368F46889
:103D800010D0FCD801E3DB2A79D963EF1AF0010ED9
:103D9000DBCF00F0020EDBCF01F000C0F3FF01C06B
:103DA000F4FF3B0EE15C02E2E16AE552E16ECBD04A
:103DB00029D9020EC9EF1FF061D90800F550DF6E56
:103DC0001200200EE66E080E39EF20F054EC2DF0B4
:103DD000E552E552E552F3CF00F0F4CF01F00001D7
:103DE000F31C1200006E016AD950010F4DD900502A
:103DF000EE260150ED221200045E000E055AF70E69
:103E000004C0DBFFF80E05C0DBFF04C0E9FF05C0FE
:103E1000EAFF1200DBCFF4FFF350F45C1200DB503A
:103E2000E76E040EE7CFDBFF12000A0EDBCF00F0D7
:103E30000B0EDBCF01F00C0EDBCF02F00D0EDBCF53
:103E400003F000500110021003101200130EEECF09
:103E5000DBFF140EEDCFDBFF130EDBCF00F0140EF3
:103E6000DBCF01F00001800E01141200F70EDBCF52
:103E700004F0F80EDBCF05F01200050EDB50E66E05
:103E8000D950130F01D9E552E750EE6EED6A1200DA
:103E90000A0EDBCF1EF00B0EDBCF1FF00C0EDBCFBC
:103EA00020F00D0EDBCF21F01200DBCFE6FF150E68
:103EB000DBCFE6FF050EDB50E552E724E552E724B1
:103EC0001200DB50CED8010EF36E060EF3CFDBFFEF
:103ED0001200EE50EFCFEAFFE96E02C0EEFF03C022
:103EE000EEFF04C0EEFF1200D9CFE6FFDACFE6FF07
:103EF000E1CFD9FFE2CFDAFF1200DFCFE6FFE66ABB
:103F00004AEC2EF0E552E552F3501200E76E080E2F
:103F1000E7CFDBFF1200EECF00F0EECF01F0EFCFE6
:103F200002F0036A1200050EDBCF00F0150EDB5025
:103F3000D88000541200010EDBCF02F0020EDBCF5E
:103F400003F0046A1200E552E5CFDAFFE7CFD9FFAC
:103F500012000A0E00C0DBFF0B0E01C0DBFF1200D7
:103F6000D9500A0F44EF20F0F36E070EF3CFDBFFBA
:103F70001200EECF00F0EFCF01F01200010EDB2AAD
:103F8000020E1200FC0EDBCFE6FFFD0EDBCFE6FFDC
:103F90001200005E000E015AF70E00C0DBFFF80EA3
:103FA00001C0DBFF00C0E9FF01C0EAFF1200DA2018
:103FB000EA6EEF2AEECFF6FF000EEF22EECFF7FF0C
:103FC000EF22EECFF8FF1200040EDBCFE6FF130E58
:103FD000DB50E552E75C9ADFDB5004DF060EDB5076
:103FE0001200090EDB500A0DF350DF24D00FE76EEC
:103FF000090EE7CFDBFFDCEF1EF0DB50F36E050EA2
:104000000AEF1FF0F70EDBCF00F0F80EDBCF01F068
:104010001200DFCFE6FFE6EF1EF028DF030EECDE36
:104020008BEF1FF038EC1AF0E552E552E552E552FD
:1040300000091200BDDEEE50EFCFEAFFE96E010E7F
:104040001200130EDB50F36E040E0AEF1FF0040E85
:10405000DB50F36E090E0AEF1FF0DBCFE6FFE6EF51
:104060001EF0E76E050EE7CFDBFF12008BDF09EFD6
:1040700020F0DBCFE6FF86DF12EF20F0D950F90FFA
:10408000E96EFF0ED7EF1FF0E96E000EDA20EA6E40
:0240900012001C
:0E409200199E08D0199E21AE05D0206C211E6B
:1040A000E86A2122198E21C01BF020C01AF02B6A69
:1040B0002A6A8E0E1C6E1D6A04EF23F0199E0CD026
:1040C000199E21AE09D01E6C1F1E201E211EE86AFB
:1040D0001F2220222122198E21C01BF020C01AF09D
:1040E0001FC02BF01EC02AF09E0E1C6E1D6A04EF2E
:1040F00023F0277E196A40EC23F058EC23F019B620
:10410000E8EF22F019A20AD019AA03D019BEE8EFED
:1041100022F019A4F4EF22F0F1EF22F019AA05D051
:1041200019ACF4EF22F0F1EF22F019A00AD019A88F
:1041300008D019BE04D019A402D0FDEF22F001EF7F
:1041400023F02A6A1D6A2750225C296E10E31FC0E3
:104150002BF020C01AF021C01BF022C028F024C090
:104160001FF025C020F026C021F0193A09D024C044
:104170002BF025C01AF026C01BF027C028F0296CB0
:10418000199E19BC198E28C01CF019B030EF23F00D
:104190001A0E296030EF23F01C6A226A19A408D095
:1041A0001F6C201E211E221EE86A202221222222AC
:1041B00019AC08D02B6C1A1E1B1E1C1EE86A1A2292
:1041C0001B221C221E6A295207E02234213220328F
:1041D0001F321E32292EF9D71F502B2620501A22AB
:1041E00021501B2222501C221EC02AF0199E1CAEF8
:1041F0000BD02A6C2B1E1A1E1B1E1C1EE86A2B22BB
:104200001A221B221C22198E1CA006D0D8801B3219
:104210001A322B322A32282A28C01CF004EF23F04D
:10422000196A40EC23F058EC23F019B6E8EF22F0BD
:1042300019A205D019BAE8EF22F0EFEF22F019BA6F
:10424000FBEF22F019A005D019B8E8EF22F0FBEF40
:1042500022F019B8EFEF22F01D6A7F0E22241C6EA7
:10426000E86A1D2227501C5EE86A1D5A1A0E286E45
:10427000226A2A6A2B6A1A6A1B6A24501F5E25501A
:10428000205A2650215A000E225A09E724501F2690
:104290002550202226502122000E222201D02A8AD7
:1042A000D8901F36203621362236D8902A362B3623
:1042B0001A361B36282EE1D7215020101F10D8A403
:1042C0002A8A04EF23F0196A40EC23F058EC23F01B
:1042D00019B6E8EF22F019A205D019B8E8EF22F0DC
:1042E000EFEF22F019AA05D019B0E8EF22F0EFEFB6
:1042F00022F019B002D019A802D0FBEF22F01D6AFB
:10430000275022241C6EE86A1D227E0E1C5EE86A7D
:104310001D5A2A6A2B6A1A6A1B6A26502102F4CF98
:104320001BF0F3CF1AF025502102F3502B26F45046
:104330001A22000E1B2226502002F3502B26F45086
:104340001A22000E1B2224502102F3502A26F45078
:104350002B22000E1A221B2225502002F3502A265F
:10436000F4502B22000E1A221B2226501F02F3505B
:104370002A26F4502B22000E1A221B22245020023F
:10438000F4502A26000E2B221A221B2225501F022F
:10439000F4502A26000E2B221A221B2204EF23F0AF
:1043A00021C02BF020C02AF020502502F4CF1FF0AE
:1043B000F3CF1EF021502602F4CF21F0F3CF20F0EE
:1043C0002502F3501F26F4502022E86A21222A50A9
:1043D0002602F3501F26F4502022E86A212226AE3E
:1043E000F6EF21F02A50205E2B50215A2BAE000C04
:1043F0002550205E2650215A000C20C02AF0205063
:104400002502F4CF1FF0F3CF1EF021502602F4CF87
:1044100021F0F3CF20F02502F3501F26F450202284
:10442000E86A21222A502602F3501F26F450202247
:10443000E86A2122000C196A40EC23F019B625EF36
:1044400022F019A20ED019B405D07F0E216EFF0EF6
:10445000206E1FD0800E216E206A1BD0216A206A38
:1044600018D019B0FBD78F0E2260EDD77E0E2264D4
:10447000F5D78E0E225C05E0D89021322032222A18
:10448000F8D719A406D0206C211EE86A212221AE9B
:10449000E5D71200196A40EC23F019B654EF22F068
:1044A00019A20FD019B407D07F0E216EFF0E206E17
:1044B0001F6E1E6E25D0800E216E01D0216A000E67
:1044C000F6D719B0FBD71E6A9F0E2260EBD77E0E7F
:1044D0002264F4D79E0E225C07E0D890213220326D
:1044E0001F321E32222AF6D719A40AD01E6C1F1EB4
:1044F000201E211EE86A1F222022212221AEDED7A3
:10450000120093EC22F019B6000C19B0000C19B48B
:10451000000C010C93EC22F019B6000C19B0000C41
:1045200019A4000C010C196A40EC23F058EC23F09C
:1045300019B6120019AE08D019A004D019A802D0DB
:1045400019801200199012002750225C0BE12650AE
:10455000215C08E12550205C05E124501F5C02E14C
:1045600019801200D8A002D0198E10D0225027C076
:1045700022F0276E215026C021F0266E205025C043
:1045800020F0256E1F5024C01FF0246E2750225C9F
:1045900010E0FF0F09E0199019B403D019AE198487
:1045A000120019AE19941200272AD890263225320B
:1045B000243224501F5E2550205A2650215A21BEF5
:1045C000EAD7D8901F3620362136222EF8D7C8D702
:1045D0007F0E226EFF0E216E206E1F6E12007F0E68
:1045E00019BEFF0E226E02D07F0E226E800E216E4B
:1045F000206A1F6AF3D719AE04D0800E226E216A9A
:10460000F7D7226A216AF4D71B501A102B102A10F0
:10461000F8E01DBEF0D71BBE0CD01C501D10EBE007
:10462000D8902A362B361A361B361C06D8A01D0603
:10463000F2D71D50D4E11C28D2E02AAE11D07F0E53
:104640002A1402E12BA00CD02B2AE86A1A221B2282
:1046500007E3D8801B321A322B321C2A1C28BFE0F9
:104660001C50C9E02BC01FF01AC020F01B34216E73
:104670001C30226E2132229E19BE228EEEEF22F0D5
:104680002136223602E31984197E06E11980226A56
:10469000216A206A1F6A1200222803E0D880213292
:1046A0001200D890213202E11982120019861200FC
:1046B0002636273602E3198C197E06E11988276A07
:1046C000266A256A246A1200272803E0D880263249
:0C46D0001200D8902632EAE1198A12008C
:0446DC00FF0EE3CF1B
:1046E000EAFFE552FF0EE3CFE9FFE552E66AE66A2C
:1046F000D9CFE6FFDACFE6FFFC0EE124D96EFF0E3C
:10470000E220DA6EE66AE66AE66A200EEF5C06E010
:10471000090EEF5C03E0EF6603D03FD0EE50F5D713
:104720002D0EEF5C03E1FF0EE32A03D02B0EEF5CAE
:1047300001E1EE502F0EEF6424D03A0EEF6021D04D
:10474000D890F90EE336FA0EE336FD0EDECFE3FF26
:10475000FE0EDDCFE3FFD890F90EE336FA0EE33616
:10476000D890F90EE336FA0EE336FD0EE350DE265E
:10477000FE0EE350DD22300EEE5CDE26000EDD2262
:10478000D9D7FF0EE3CFE8FFE85207E0F90EE31EAA
:10479000E32AFA0ED8B4E306E31EE552E552E552E9
:1047A000FF0EE3CFDAFFE552FF0EE3CFD9FFE5526C
:1047B000E1CFE9FFE2CFEAFFED52ED52EECFF3FF9A
:1047C000EFCFF4FF1200D9CFE6FFDACFE6FFE66ABB
:1047D000E66AE66AE66AE66AE66AE66AE66AE66A59
:1047E000E66AF20EE3CFE9FFF30EE3CFEAFF200E15
:1047F000EF5C06E0090EEF5C03E0EF6603D07BD0D0
:10480000EE50F5D72D0EEF5C03E1FF0EE38003D0F1
:104810002B0EEF5C01E1EE50FA0EE124D96EFF0E93
:10482000E220DA6E2E0EEF5C04E1FF0EE382EE5220
:10483000F9D72F0EEF6449D03A0EEF6046D0D890EA
:10484000FA0EE336FB0EE336FC0EE336FD0EE336DE
:10485000F60EDECFE3FFF70EDECFE3FFF80EDECF7E
:10486000E3FFF90EDDCFE3FFDD52DD52D890FA0E03
:10487000E336FB0EE336FC0EE336FD0EE336D8904E
:10488000FA0EE336FB0EE336FC0EE336FD0EE3369E
:10489000F60EE350DE26F70EE350DE22F80EE3506C
:1048A000DE22F90EE350DD22DD52DD52300EEE5CE9
:1048B000DE26000EDE22DE22DD22DD52DD52FF0E7C
:1048C000E3A2B0D7FE0EE306ADD7FF0EE3A013D0F0
:1048D000FA0EE31EFB0EE31EFC0EE31EFD0EE31EAE
:1048E000FA0EE32A08E1FB0EE32A05E1FC0EE32AB7
:1048F00002E1FD0EE32AF20EE9CFE3FFF30EEACF69
:10490000E3FFEE0EE3CFD9FFEF0EE3CFDAFFFA0EAF
:10491000E3CFDEFFFB0EE3CFDEFFFC0EE3CFDEFFD7
:10492000FD0EE3CFDDFFDD52DD52F00EE3CFD9FF08
:10493000F10EE3CFDAFFFE0EE3CFDFFFF20EE1244C
:10494000E96EFF0EE220EA6EF60EE126FF0EE2228D
:10495000FF0EE3CFDAFFE552FF0EE3CFD9FFE552BA
:10496000EECFF3FFEFCFF4FF1200D9CFE6FFDACF9F
:10497000E6FFFA0EE3CFD9FFFB0EE3CFDAFFFD0E21
:10498000E35209E72D0EDE6EFC0EE31EE32AFD0E58
:10499000D8B4E306E31EE652E652E652FD0EE124E9
:1049A000E76EFF0EE220E46EE652F70EE3CFE6FF7D
:1049B000F70EE3CFE6FF25EC25F0F90EE124E96ED2
:1049C000FF0EE220EA6E15EC25F00AE112EC25F06C
:1049D00009E115EC25F008E112EC25F007E108D01B
:1049E00020EC25F01BEC25F020EC25F01BEC25F04D
:1049F00020EC25F0DE6AF90EE126FF0EE222FF0E22
:104A0000E3CFDAFFE552FF0EE3CFD9FFE552FC0E0C
:104A1000E124E96EFF0EE220EA6EEECFF3FFEFCF66
:104A2000F4FF1200EF380F0B1200EF500F0B02E1F2
:104A3000EE52D8841200EF380F0B300FDE6E1200EA
:104A4000EE500F0B300FDE6E1200FC0EE3CFE9FFCD
:104A5000FD0EE3CFEAFF100EE66EEE6AEE6AEF6A35
:104A6000D890FD0EE336FE0EE336ED36ED36EF362A
:104A7000FF0EE30609E046EC25F0EE5246EC25F089
:104A8000EE5246EC25F0EDD7E56E1200030EEF2452
:104A9000E8B6EF6E300EEF24E8BEEF6E000CD9CF13
:104AA000E6FFDACFE6FFF80EE3CFD9FFF90EE3CF4A
:104AB000DAFFE652E652E652E652E652FB0EE124F7
:104AC000E76EFF0EE220E46EE652F30EE3CFE6FF60
:104AD000F30EE3CFE6FFF30EE3CFE6FFF30EE3CFF3
:104AE000E6FFD4EC25F0F50EE124E96EFF0EE2209E
:104AF000EA6EC1EC25F019E1C4EC25F018E1C1EC37
:104B000025F017E1C4EC25F016E1C1EC25F015E124
:104B1000C4EC25F014E1C1EC25F013E1C4EC25F060
:104B200012E1C1EC25F011E112D0CAEC25F0CFEC76
:104B300025F0CAEC25F0CFEC25F0CAEC25F0CFEC3F
:104B400025F0CAEC25F0CFEC25F0CAEC25F0CFEC2F
:104B500025F0DE6AF50EE126FF0EE222FF0EE3CF1E
:104B6000DAFFE552FF0EE3CFD9FFE552FA0EE1245A
:104B7000E96EFF0EE220EA6EEECFF3FFEFCFF4FF17
:104B80001200EF380F0B1200EF500F0B02E1EE5244
:104B9000D8841200EF380F0B300FDE6E1200EE508B
:104BA0000F0B300FDE6E1200FA0EE3CFE9FFFB0EA3
:104BB000E3CFEAFF200EE66EEE6AEE6AEE6AEE6A78
:104BC000EF6AD890FB0EE336FC0EE336FD0EE336BB
:104BD000FE0EE336ED36ED36ED36ED36EF36FF0EF2
:104BE000E3060FE003EC26F0EE5203EC26F0EE5263
:104BF00003EC26F0EE5203EC26F0EE5203EC26F026
:104C0000E1D7E56E1200030EEF24E8B6EF6E300E2A
:084C1000EF24E8BEEF6E000C7A
:084C1800000000000000005F35
:104C200000000007000700147F147F14242A7F2A45
:104C30001223130864623649552250000503000010
:104C4000001C2241000041221C0014083E081408E8
:104C5000083E0808005030000008080808080060F6
:104C600060000020100804023E5149453E00427F8A
:104C7000400042615149462141454B311814127F91
:104C80001027454545393C4A49493001710905031A
:104C90003649494936064949291E00363600000082
:104CA0005636000008142241001414141414004154
:104CB0002214080201510906324979413E7E111140
:104CC000117E7F494949363E414141227F4141227F
:104CD0001C7F494949417F090909013E4149497AF7
:104CE0007F0808087F00417F41002040413F017F4D
:104CF000081422417F404040407F020C027F7F0425
:104D000008107F3E4141413E7F090909063E41515D
:104D1000215E7F09192946464949493101017F0130
:104D2000013F4040403F1F2040201F3F4038403F50
:104D3000631408146307087008076151494543006C
:104D40007F41410002040810200041417F0004021D
:104D5000010204404040404000010204002054543D
:104D600054787F48444438384444442038444448C4
:104D70007F3854545418087E0901020C5252523E96
:104D80007F0804047800447D40002040443D007FBB
:104D90001028440000417F40007C041804787C08FF
:104DA00004047838444444387C1414140808141457
:104DB000187C7C080404084854545420043F4440A0
:104DC000203C4040207C1C2040201C3C4030403C8B
:104DD00044281028440C5050503C4464544C440027
:104DE0000836410000007F0000004136080010082E
:104DF0000810087846414678436D6420004E756D72
:104E0000200044726F6974650047617563686500CE
:104E1000566F6C2E2B2000566F6C2E2D20004F4BA2
:104E2000004D656E7520004D75746520004F7364EC
:104E300020004861757420004261732000436C6556
:104E4000617220004D656D6F2000436F7272656363
:104E5000742000736C656570200041696775202BB4
:104E6000200041696775202D2000706F696E740005
:104E70002020202020202020202020202020202032
:104E80002000506F727420636F6D6D2031393230A5
:104E900030206F75766572740050524F4A45543A0F
:104EA000203138463235785F4444535F49525F6160
:104EB0006C6C2E6D63700D0045534320706F7572DE
:104EC00020736F727469720D004D4152414E545AF5
:104ED0002052433532303053520D00202020202004
:104EE000202020202020202020202020200D0063B2
:104EF00061722072656375203A00202020202020F6
:104F00002020202020202020202020200D002020D4
:104F10002020202020202020202020202020202091
:104F20000D002020200D0020200D00495220545358
:104F30004F50333620436170747572653D200D000B
:104F40003138463235385F4444535F414439383351
:104F5000355F4C4344333331305F52733233325F09
:104F6000495243355F3131313032325F616C6C2EE2
:104F7000630D00313846323538204E6F6B69612041
:104F80004C434400496E69742044445320414439E1
:104F9000383335200046726571303D20332E303075
:104FA00030487A20200046726571313D2031302E24
:104FB00030303030487A0053616973696520467239
:104FC000657175656E63650054534F5033362043E9
:104FD0006170747572653A00456E74726572207600
:104FE000616C657572203A200078787878787878E6
:104FF000782E787820487A202000537765657020D5
:1050000031302D3230303030487A002E2E2E2E2E78
:0C5010002E2E2E2E2E2E2E2E2E2E2E009A
:04501C00D9CFE6FF03
:10502000DACFE6FFE1CFD9FFE2CFDAFF100EE124BD
:1050300002E3E168E652E16E0F0EDB6AD950020F1F
:10504000E66E000EDA20E66ED950060FE66E000E10
:10505000DA20E66EFC0EDBCFE6FFFD0EDBCFE6FFCF
:10506000E3EC23F0006E060EE15C02E2E16AE55239
:10507000E16E0050F3CFDEFFF4CFDDFFDECFE9FFBE
:10508000DDCFEAFFEF50DF0B450814E1DF2A010E08
:1050900001E3DB2ADECFE6FFDDCFE6FF6EEC23F097
:1050A000E552E552060EDBCFE7FFF350E726060E8A
:1050B000E7CFDBFF020EDBCF00F0030EDBCF01F00A
:1050C000040EDBCF02F0050E03D960EC20F0F3D81C
:1050D000060EDB5001E190D006D900340BE3010E3F
:1050E000F36E0F0EF3CFDBFF060EDB50FF0D060E47
:1050F000F3CFDBFF0B0EDB6A0C0EDB6A800EF36E68
:105100000D0EF3CFDBFF3F0EF36E0E0EF3CFDBFF82
:10511000EAD8140EE76E0018E8AE02D0E73402D0E9
:10512000E750005C0BE397D8EC0E246E780E256EEA
:10513000AD0E266E600E77D8140EB3D8D4D80A0EF2
:10514000E76E0018E8AE02D0E73402D0E750005C0A
:105150000BE381D8F90E246E020E256E150E266E15
:10516000500E61D80A0E9DD8BED8050EE76E001805
:10517000E8AE02D0E73402D0E750005C0AE36BD817
:10518000246A500E256EC30E266E470E4CD8050EAF
:1051900088D8A9D8020EE76E0018E8AE02D0E7342E
:1051A00002D0E750005C09E356D8246A256AC80E8D
:1051B000266E420E38D8020EEBD795D8010EE76E58
:1051C0000018E8AE02D0E73402D0E750005C09E3F3
:1051D00042D8246A256A200E266E410E24D8060E77
:1051E000DB060F0EDB5004E043D810EC21F003D0B7
:1051F0003FD863EC21F05FD8070EDBCF00F0080E3C
:10520000DBCF01F0090EDBCF02F00A0E61D8100EE1
:10521000E15C02E2E16AE552E16EE552E5CFDAFFD8
:10522000E7CFD9FF1200276E00C01FF001C020F0A9
:1052300002C021F003C022F063EC21F00B0E1FC06E
:10524000DBFF0C0E20C0DBFF0D0E21C0DBFF0E0EBE
:1052500022C0DBFF12000B0EDBCF00F00C0EDBCF09
:1052600001F00D0EDBCF02F00E0EDBCF03F01200CB
:10527000070EDBCF1FF0080EDBCF20F0090EDBCFCF
:1052800021F00A0EDBCF22F00B0EDBCF24F00C0E48
:10529000DBCF25F00D0EDBCF26F00E0EDBCF27F097
:1052A0001200006E060EDBCFE7FF0050E75E060E31
:1052B000E7CFDBFF1200070E1FC0DBFF080E20C088
:1052C000DBFF090E21C0DBFF0A0E22C0DBFF12004C
:1052D000DBCF03F000C01EF001C01FF002C020F0C1
:0E52E00003C021F01200060EDBCF00F012001A
:0252EE00D9CF16
:1052F000E6FFDACFE6FFE1CFD9FFE2CFDAFF130E08
:10530000E12402E3E168E652E16E0C0EDB6AD9505B
:10531000FA0FE96EFF0EDA20EA6E080EEECFDBFF21
:10532000090EEECFDBFF0A0EEECFDBFF0B0EEECF4A
:10533000DBFF1FD9D950080F17D9EECFE6FFEECF0C
:10534000E6FFEECFE6FFEFCFE6FFC0EC2AF0006EFF
:10535000060EE15C02E2E16AE552E16E0050DF6EAA
:10536000020EDF5C01E0BCD0050EDBCF02F0060EC2
:10537000DBCF03F0F80EDB50025C006EF90EDB5061
:105380000358016E7F0E005E000E015A0D0E00C024
:10539000DBFF0E0E01C0DBFF0D0E0E0EDBCF01F0AA
:1053A0000001800E01140AE0010EF36E0C0EF3CF23
:1053B000DBFF070EDB5001E098D09DD00D0EDBCF58
:1053C00000F00E0EDBCF01F0D890015004E6170E6E
:1053D000005C000E015801E39ED0046805687F0E52
:1053E000066E076A0D0EDB501F0B04C000F005C0EF
:1053F00001F006C002F007C003F007E0D8900332C6
:10540000023201320032E806F9E10F0E00C0DBFF84
:10541000100E01C0DBFF110E02C0DBFF120E03C035
:10542000DBFF0F0EDBCF00F0100EDBCF01F0110E13
:10543000DBCF02F0120EDBCF03F0D950010F94D86E
:10544000EE500016EE500116EE500216EE50031606
:10545000005001100210031002E1000E01D0010EF5
:10546000E76E0C0EE7CFDBFFDB5055E0046A056A00
:10547000800E066E076A010E086E096A0A6A0B6AD8
:10548000D9500F0F71D8EE500826EE500922EE5079
:105490000A22EE500B220850045C006E0950055899
:1054A000016E0A500658026E0B500758036ED95011
:1054B000010F5AD80050EE160150EE160250EE16AB
:1054C0000350EE16D950080FE66E000EDA20E66E95
:1054D00050D84EEC2BF0E552E552E552E5521BD088
:1054E000DF0419E1070EDB5006E0006A016A026A78
:1054F000800E036E04D0006A016A026A036A080E15
:1055000000C0DBFF090E01C0DBFF0A0E02C0DBFF9B
:105510000B0E03C0DBFFF60EDBCFE9FFF70EDBCF90
:10552000EAFF0C0EDBCFEFFF080EDBCF00F0090E19
:10553000DBCF01F00A0EDBCF02F00B0EDBCF03F066
:1055400000C01EF001C01FF002C020F003C021F017
:10555000130EE15C02E2E16AE552E16EE552E5CF4D
:10556000DAFFE7CFD9FF1200E96E000EDA20EA6E0B
:105570001200D950010FE66E000EDA20E66E12001E
:10558000D9CFE6FFDACFE6FFE1CFD9FFE2CFDAFFEE
:10559000E652006801687F0E026E036AD950FA0F66
:1055A000E96EFF0EDA20EA6EEE500016EE5001169C
:1055B000EE500216EE5003166AD800C0EEFF01C08E
:1055C000EEFF02C0EEFF03C0EEFFFD0EDB50800BCE
:1055D00002E0010E01D0000EE66E59D8060EE92653
:1055E000000EEA22E552E750EF6EFC0EDBCF00F032
:1055F000FD0EDBCF01F0D89000360136FC0E00C066
:10560000DBFFFD0E01C0DBFFDB50E66E40D8040E71
:10561000E926000EEA22E552E750EE6EED6AFD0E35
:10562000DB50006E016AFF0E001818E1015016E110
:105630002ED8EECF00F0EECF01F0EECF02F0EFCF9C
:1056400003F0005001100210031006E0210E0101CA
:10565000B56FB66B800E0BD0040E09D0FD0EDB507B
:1056600008E115D8EE6AEE6AEE6AEE6A010EDF6EA8
:1056700006D0020EDF6E0BD8EE52EE52EE8EDF50E9
:10568000E552E552E5CFDAFFE7CFD9FF1200F80E79
:0C569000DBCFE9FFF90EDBCFEAFF1200D0
:04569C00D9CFE6FF7D
:1056A000DACFE6FFE1CFD9FFE2CFDAFF5BD80134F2
:1056B00011E20050FE08000E01540CE276D805E01D
:1056C0006CD8800EEE6EEE6847D067D8800EEE6E16
:1056D0007F0E0ED047D8D890015004E6010E005C32
:1056E000000E01580BE261D805E057D8EE6A800E33
:1056F000EE6E32D052D8EE6AEE6A2ED047D8EECF98
:1057000000F0EECF01F0EECF02F0EFCF03F032D891
:1057100000C0EEFF01C0EEFF02C0EEFF03C0EEFFCF
:1057200021D80050010B05E025D8020E3AD8EF8EA3
:1057300004D020D8020E35D8EF9E14D8D89001326C
:10574000003218D8030E2DD800C0EFFF1AD804E09D
:1057500011D8030E26D8EF8EE552E5CFDAFFE7CF5A
:10576000D9FF120013D8040E1CD8EECF00F0EFCFF3
:1057700001F01200FA0EDBCFE9FFFB0EDBCFEAFFF0
:10578000120004D8060E0DD8EF501200FC0EDBCF2D
:10579000E9FFFD0EDBCFEAFF1200ECDFEE6AEE6AF6
:1057A0001200E926000EEA221200220E0101B56F56
:0657B000B66BC1EF2BF007
:0A57B600D9CFE6FFDACFE6FFE1CF1E
:1057C000D9FFE2CFDAFF060EE12402E3E168E652F8
:1057D000E16ED950050FE66E000EDA20E66E000E7F
:1057E000E66EE66AD950FA0FE96EFF0EDA20EA6E2D
:1057F000EECFE6FFEECFE6FFEECFE6FFEFCFE6FF20
:1058000077EC29F0006E080EE15C02E2E16AE552F5
:10581000E16E0050010E1EC0DBFF020E1FC0DBFF59
:10582000030E20C0DBFF040E21C0DBFF050EDB50A2
:105830002AE0040EDB50800B26E1006A016A800E2C
:10584000026E3F0E036ED950010FE96E000EDA2092
:10585000EA6EEECF1FF0EECF20F0EECF21F0EFCFCB
:1058600022F000C024F001C025F002C026F003C0E1
:1058700027F07AEC20F022C0EDFF21C0EDFF20C020
:10588000EDFF1FC0EFFF010EDBCF00F0020EDBCFFC
:1058900001F0030EDBCF02F0040EDBCF03F000C0FB
:1058A0001EF001C01FF002C020F003C021F0060E60
:1058B000E15C02E2E16AE552E16EE552E5CFDAFF32
:0658C000E7CFD9FF120042
:0A58C600D9CFE6FFDACFE6FFE1CF0D
:1058D000D9FFE2CFDAFFE652E652E652E652D9505D
:1058E000F90F006EFF0EDA20016E020E00C0DBFF22
:1058F000030E01C0DBFF020EDBCFE6FF030EDBCFA2
:10590000E6FFF90EDBCFE6FFFA0EDBCFE6FFFB0E7C
:10591000DBCFE6FFD950FC0FE66EFF0EDA20E66E15
:105920004EEC1AF0006E070EE15C02E2E16AE5520D
:10593000E16E0050F3CFDEFFF4CFDDFFFC0EDBCFD6
:10594000E9FFFD0EDBCFEAFFEF6ADECF00F0DDCF2F
:1059500001F000C0F3FF01C0F4FF040EE15C02E2BD
:10596000E16AE552E16EE552E5CFDAFFE7CFD9FF14
:02597000120023
:0E5972001E0EF66E000EF76E000EF86E0101AE
:105980000900F550B06F0900F550B16F03E1B06741
:1059900001D03DD00900F550AB6F0900F550AC6F58
:1059A0000900F550AD6F09000900F550E96E0900D6
:1059B000F550EA6E090009000900F550AE6F0900C4
:1059C000F550AF6F09000900F6CFB2F1F7CFB3F190
:1059D000F8CFB4F1ABC1F6FFACC1F7FFADC1F8FF32
:1059E0000101AE5302E1AF5307E00900F550EE6E3E
:1059F000AE07F8E2AF07F9D7B2C1F6FFB3C1F7FFC0
:105A0000B4C1F8FF0101B007000EB15BBFD71200AF
:105A1000FB0EE3CFF6FFFC0EE3CFF7FFFD0EE3CF67
:105A2000F8FFFE0EE3CFE9FFFF0EE3CFEAFFE9CF79
:105A3000F3FFEACFF4FF0900F5CFEFFFEE66FBD7E7
:105A40001200FE0EE3CFE9FFFF0EE3CFEAFFF36A99
:105A5000F46AEE5203E0F34AF42AFBD71200FF0E79
:105A6000E3CFF8FFE552FF0EE3CFF7FFE552FF0E5D
:105A7000E3CFF6FFE552E66AE66AE66A0900F55208
:105A800009E0FD0EE32A05E1FE0EE32A02E1FF0E26
:105A9000E32AF4D7FD0EE3CF1FF0FE0EE3CF20F094
:085AA000FF0EE3CF21F012001C
:085AA800D9CFE6FFDACFE6FFDB
:105AB000E1CFD9FFE2CFDAFFFB0EDBCF00F0FC0E27
:105AC000DBCF01F00001800E01141AE1FB0EDBCFE9
:105AD000E9FFFC0EDBCFEAFFEECFF3FFEDCFF4FFE3
:105AE000EE2A000EEF22F3CFE9FFF4CFEAFFFD0E1E
:105AF000DBCFEFFFEF50016AF36E01C0F4FF10D06F
:105B0000FB0EDB50FE0806E1FD0EDBCFE6FF7AEC74
:105B10002EF005D0FD0EDBCFE6FF03EC00F0E552E2
:0C5B2000E552E5CFDAFFE7CFD9FF120015
:045B2C001E502302E2
:105B3000F3CF1AF0F4CF1BF02402F3501B26000E13
:105B4000F4201C6E1E502502F3501C26000EF4207B
:105B50001D6E1E502602F3501D261F502302F350C7
:105B60001B26F4501C22000E1D221F502402F3504D
:105B70001C26F4501D221F502502F3501D262050D4
:105B80002302F3501C26F4501D2220502402F3500F
:0C5B90001D2621502302F3501D26120098
:045B9C00D9CFE6FF78
:105BA000DACFE6FFE1CFD9FFE2CFDAFFF292FD0EC6
:105BB000DBA202D0F18C01D0F19CDBA002D0F18EEF
:105BC00001D0F19E9380DBAC02D0F18001D0F19046
:105BD000DBAE02D0F28801D0F298E552E5CFDAFFD1
:065BE000E7CFD9FF12001F
:0A5BE6001D6A1C6A1B6A1A6A200E71
:105BF000E76ED8901E361F36203621361A361B36F1
:105C00001C361D3623501A5C24501B5825501C5836
:105C100026501D5809E323501A5E24501B5A255064
:0E5C20001C5A26501D5A1E2AE72EE4D71200E9
:025C2E00D9CFCC
:105C3000E6FFDACFE6FFE1CFD9FFE2CFDAFFFD0ED4
:105C4000DB507F0BD56ED76AD66AF294FD0EDBAEC1
:105C500002D0F28A01D0F29AD58EE552E5CFDAFF72
:065C6000E7CFD9FF12009E
:0A5C6600FF0EE3502F6EEF0E01D089
:105C7000F30EE76EE72E3AEF2EF00C0E2E6EE76A6B
:105C8000E72E40EF2EF02E2E3FEF2EF02F2E38EF86
:045C90002EF01200E0
:0C5C9400F36AF46AFF0EE124E96EFF0ED3
:105CA000E220EA6EED6607D02F0EEF6404D03A0EC4
:085CB000EF6001D0F32A12009D
:085CB800000EF36E00EE00F097
:105CC000060E01D81200EA6002D0EE6AFCD7F3504B
:085CD000E9601200EE6AFCD746
:085CD80015EE00F025EE00F0CE
:105CE000F86A199CB9EC2CF091EC2EF06EEC14F0E3
:045CF000FBD71200CC
:0C5CF400FF0EE350ACBA04D0AF6AAB8ED8
:105D0000AC8A949CACA2FED7AD6EF36EF46A12001E
:105D10003031323334353637383961626364656621
:015D20000082
:025D220012006D
:0C5D24002E2E2E2E2E2E2E2E2E2E2E2E4B
:105D30002E2E2E2E2E2E2E2E2E2E2E2E2E2E2E2E83
:105D40002E2E2E2E2E2E2E2E2E2E2E2E2E2E2E2E73
:105D50002E2E2E2E2E2E2E2E2E2E2E2E2E2E2E0091
:105D60000000000030303030303030300000023180
:105D70003233343536373839303132333435003117
:105D80003233343536373839303132333435360002
:105D90000000000000000000000000000000000003
:105DA00000000000000000000000000000000000F3
:105DB00000F84DFD4D024E094E104E174E1E4E215D
:105DC0004E274E2D4E324E384E3D4E444E4A4E5387
:105DD0004E5A4E624E6A4E0D0F10111718191C1DA7
:105DE0002226292B2C2E313C00080904050610110F
:105DF0000A0B0E0F120203070C0D00704E824E9913
:105E00004EB84EC94EDB4EEF4EFA4E0E4F224F2784
:105E10004F2B4F404F734F844F954FA64FB74FC8EE
:095E20004FD84FE94FFA4F0B5027
:020000040030CA
:01000100FA04
:01000200F409
:01000300FEFE
:01000600FBFE
:0200000400F00A
:10000000506F727420436F6D20313932303062206E
:100010002620496E697420484152442E2E2E0D0030
:100020002E2E2E2E2E2E2E2E2E2E2E2E2E2E2E2EF0
:1000300020203C4553433E206578697420200D0004
:100040002E2E2E2E2E2E2E2E2E2E2E2E2E2E2E2ED0
:100050002E2E2E2E2E2E2E2E2E2E2E2E2E2E0D000F
:1000600055736167652049326320536F6674776109
:100070007265204D504C41422043313820200D0004
:10008000313846323538206176656320626F6F748F
:100090006C6F6164657220202020202020200D00DC
:1000A0007061756C666A756A6F40667265652E660A
:1000B00072202020202020202020202020200D0021
:1000C0004D504C4142204944452056382E36332E5F
:1000D0002E2E2E2E2E2E2E2E2E2E2E2E2E200D009D
:1000E0004D504C4142204331382076332E33372E49
:1000F0003031202E2E2E2E2E2E2E2E2E0D0A0000CA
:00000001FF
